:10000000F01F0010294F0000274F0000274F00006D
:10001000274F0000274F0000274F0000000000007E
:10002000000000000000000000000000274F00005A
:10003000274F000000000000274F0000FD210000B6
:10004000052000000520000005200000052000001C
:10005000052000000520000005200000052000000C
:1000600005200000052000000520000005200000FC
:1000700005200000254F0000254F0000C1000000B2
:10008000C5220000DD220000F12400000925000047
:10009000254F00004D260000254F0000254F000091
:1000A000254F0000254F0000254F0000254F000080
:1000B000254F0000254F0000254F0000254F000070
:1000C000554B10B51A6801321A60544B1A68544BDC
:1000D000D2B2302A69D01ADC182A44D012DC082A9D
:1000E00032D0102A00D094E04E4A002111604E49CF
:1000F0000A68501C08604D49895C4D4AC9B21160BC
:10010000282287E0202A63D0282A32D081E0482A9A
:100110005ED004DC382A51D0402A53D079E0502AEE
:1001200060D0582A75D13F490A68501C0860404980
:1001300008684049C0B288543F4A0221FF3111602B
:1001400080221021D20563E0374A00211160116836
:10015000481C1060354A515C354AC9B211602822EA
:100160001A6001223CE030490A68501C08602F499F
:1001700009E02D4A314910680968884207D21168A0
:10018000481C1060294A515C294AC9B240E02C4AF7
:1001900011688022D205002901D0202138E02649AB
:1001A0000220FF300860102132E08022D2051021A9
:1001B000116008221A608122520011E08221490058
:1001C0001D4A25E01E4A1168042201291AD11DE0AA
:1001D0008022D2051021116008221A600422FF3209
:1001E000154B17E00F4A1168481C1060104804684E
:1001F0001048E4B244541068114A116804220139CD
:10020000884203D28021C9050A6002E01A6000E03A
:10021000116008221A6010BD88020010040000401E
:10022000180000407C020010840200109C040010A2
:10023000080000408C04001080020010AC04001084
:10024000880400101B4B02211A6810B50A431A607B
:10025000194B20211A68041C0A431A60174B1849CD
:100260001A680A401A601868012210431860154B7A
:1002700018680140196019680A431A60124B6C2211
:100280001A60124B1249186804F0D4FE114A10602B
:10029000114A1060022C02D1104BA0221A60104BA0
:1002A000802212021A6080234022DB0501201A609E
:1002B00010BDC046048004408080044030400440AB
:1002C000F8FCFFFF34400440180000408004001098
:1002D000400D030014000040100000400C000040DE
:1002E00000E100E0034B1B689A06FBD5024B186047
:1002F0007047C0461480004000800040FFFFFFFFB1
:1003000070B5061C00200D1C01F06CF9002801D00E
:1003100002F072FD00242C60301C3460291C01F0B6
:100320008FF9201C01F05EF9A04207D002F064FDB5
:100330002C60301C3460291C01F082F970BD08B5B6
:1003400001F08CFF08BD08B500230B60036001F0CD
:1003500077F908BD10B502F017FD0D4B00201968A4
:1003600002F03CF9002002F029F9002002F006F921
:10037000084B01241C60084B201C198801F0EAFF7F
:10038000201C01F0D7FF201C01F0B4FF10BDC046B7
:100390007C040010780200108404001010B50624BC
:1003A00001200021013C01F025FF002CF8D1FFF7CE
:1003B000D1FF10BD08B5002002F0F0F8012001F0D7
:1003C000A9FF02F0E7FC08BD38B5051C0C1CFFF7BF
:1003D000C1FF054B0122281C211C5A6203F0D8FFE3
:1003E000FFF7E8FF38BDC046580C001010B5041CDC
:1003F000FFF7B0FF201C03F03BFF041CFFF7DAFF00
:10040000201C10BD08B50020FFF7F0FF08BD00005C
:1004100008B5021C0249034802F03EFB08BDC04675
:10042000645100005C51000037B500F051FF032219
:10043000164B1748002101F039F800F053FFFFF781
:10044000E1FF1448FFF7E4FF134B144A00241A603D
:100450001D1C2B689C4211DA02F0DAF9002803D047
:1004600001F0A8FC00240FE00A2001F0F7FE684626
:1004700001A9FFF745FF009B002B05D0FFF7C2FF46
:10048000074802F009FB37BD0134E2E78C5A00004F
:100490006D5100007C5100006C03001070170000CB
:1004A00082510000704700001B4B73B5041C1B49B0
:1004B000186804F0BFFD1A4900901A4A1A4B201C14
:1004C00002F0F6FA01F098F9002812D001F0B0F924
:1004D000FA218900061C04F0ADFD051C201C02F069
:1004E00038FB124B20186B431149F3182A1C02F0F9
:1004F000DFFA201C02F02DFB0E4B20181B68002B8E
:1005000002D003DA0C4A02E00C4A00E00C4A0D4922
:1005100002F0CEFA73BDC0468004001040420F00C6
:100520009351000064510000A051000018FCFFFF2F
:10053000A451000048010010905100008D510000AE
:100540005D9A0000AF51000070B5051C0E1C141C14
:1005500000F0BEFE301C291C0022064B00F0A6FF56
:10056000201C01210922044B00F0A0FF00F0BAFE7C
:1005700070BDC0468C5A0000845A000000B5084B7C
:1005800089B01A78074B68461B78074902F090FA41
:1005900001206946054AFFF7D7FF09B000BDC046F4
:1005A0003C01001000000010E3510000F151000078
:1005B000F0B52A4C2A4D237885B001932F78FFF7A8
:1005C000DDFFFFF71FFF002602A803A9FFF798FE33
:1005D000029800282BD0C0B200F082FF40280CD037
:1005E00004D830280ED0392817D01BE0462830D048
:1005F00049280DD0412815D126E02B783E2B11D863
:10060000013303E02B78002B0CD0013B2B7009E069
:100610002378062B06D8013303E02378002B01D082
:10062000013B237000F040FEFFF7A8FF0026029B6D
:10063000002B02D0C82001F011FE04200321013656
:1006400001F0D8FD1D2EBFDD019B2F70237000F03F
:100650002BFEFFF7D7FE05B0F0BDC046000000102E
:100660003C01001038B5051C0C1C00F0FCFD291CD9
:10067000221C0120FFF768FF034B00225A60034A47
:10068000943212689A6038BD580C0010BC040010F7
:1006900010B590B0041C6846FFF706FF201C6946A1
:1006A0006A46FFF751FF10B010BD000000B52D22C3
:1006B0008DB0002800D02B2268460D4902F0F8F9D1
:1006C00004A802F02BFC0120694604AAFFF73CFFB6
:1006D0000320002101F08EFD0220FFF787FE002895
:1006E000EED00A20002101F085FD0DB000BDC0460E
:1006F0002452000070B58CB0FFF784FE02A81449A4
:1007000002F030FA2E25FF3504AE301C02F006FC54
:100710006846002409A90930F47402F023FA02AAF9
:100720000420311CFFF710FF201C032101F062FDA3
:10073000684601A901940094FFF7E2FD009BA342E3
:1007400002D1013DA542DFD1FFF75CFE0CB070BDC8
:100750005E9A0000F0B5002493B00594FFF752FEB6
:100760000222962301940392251C5B00029300F061
:10077000AFFD019B9A4F002B6DD10AAE301C02F0E9
:10078000CDFB019AF27432747273B272F2713271EB
:10079000002C01D1012D05D1301C042100223B1C6D
:1007A00000F084FE8F4E3B1C301C1E21002200F006
:1007B0007DFE8B4F012C01D1012D06D168462D30D5
:1007C000252100223B1C00F071FE301C3321002249
:1007D0003B1C00F06BFE824E022C09D1012D07D08C
:1007E000684633304D210022331C00F05FFE09E0E3
:1007F0000CA83A210022331C00F058FE032CEFD144
:10080000012DEDD0784F331C381C5921002200F007
:100810004DFE734E042C01D1012D06D168463630B1
:100820005F210022331C00F041FE381C6C210022A5
:10083000331C00F03BFE052C01D1012D06D168468A
:10084000393072210022664B00F030FE0FA80421DF
:100850000922664B03E06648042100223B1C00F09D
:1008600025FE00F03FFD059B002B0AD0143B012B19
:1008700005D8052C03D0962001F0F0FC01E0FFF72D
:10088000C1FD0320011C01F0B5FC5A4B1E68002E6F
:10089000F7D1301C00F0A6FE06A9071C05A8069695
:1008A0000596FFF72DFD059B002B73D007AE08AF13
:1008B000301C391C09AA02F065FB019000286FD199
:1008C000301C02F049FC051C05981238052866D832
:1008D00004F04EFB0565240C6503601C00E0601D00
:1008E000062104F0FDFB00250C1C59E0052C56D810
:1008F000201C04F03DFB03060B0D10393388013337
:1009000016E0B0780C2104F08BFB18E001355DE0B7
:10091000387801301AE0787801301FE0052C3ED895
:10092000201C04F025FB03070F1119213388013B1C
:10093000338044E0B0780C210A3004F0D1FB01315F
:10094000B1703CE0013D41E038781730182104F0E7
:10095000C7FB042239703FE078783B303C2104F03B
:10096000BFFB032379702FE00023BB70281C0721F5
:1009700004F0B6FB301C0A1C0991391C052C02D16D
:1009800002F05BFB02E0039B02F016FB01259623BD
:10099000AB4007E0002F06D101235D4003E00125B5
:1009A00096235B000293059B842B17D0182B15D040
:1009B000029B029A013B002A00D0D7E60EE0301CD1
:1009C00002F0CAFB0523051C0393CFE7281C311C4A
:1009D00002F0F2FB022405220392C7E713B0F0BD38
:1009E0008C5A00002D52000022520000845A000050
:1009F0002F52000060020010F7B502F025FA18200F
:100A00000021FFF7E1FC00246B4EFFF7D3FC6B4D98
:100A100000236B62201C02F038FA002C02D0002068
:100A2000012101E00620032101F0E4FB201C02F07B
:100A300027FA01A9071C6846002F03D0FFF783FCA3
:100A4000012728E0FFF77FFC009A002A23D1002C21
:100A5000E0D15B4F3B1C98331B68002B0DD1594BE9
:100A6000F618D7D5182000219437FFF7ADFC3C6865
:100A700063425C4100F0E0FBCCE7534B00941A6802
:100A800011321A60009A102AE9DC03F0A1FB009BE6
:100A900001330093F6E7002C0CD0009B182B01D0FB
:100AA000002FB2D000F026FC4848FFF7B1FC444BC1
:100AB0000122DA6600F0CEFE02F030F9009A182A20
:100AC00062D1019F0024F8B200F00AFD01260194D2
:100AD0006E62172846D00CD813282BD002D81128C4
:100AE00019D04EE015282DD016284AD1FFF760FD09
:100AF0004AE026282ED004D819281ED0212811D04B
:100B00003FE0442836D045283BD1E120000102F0E7
:100B1000ADFA301C32E02E4B1B68002B34D0FFF7AF
:100B2000E9FD05E02A4B1B68002B2DD0FFF712FED4
:100B3000009429E0FFF778FC26E0264B1868301A6D
:100B400000F0AEFF0120FFF7A3FDFFF75BFCFFF70E
:100B500025FC19E0204B05221C70204B1A7000F078
:100B6000A3FB11E01E4B1A6801321A60052A0BD153
:100B70001C6009E01B4802F079FA201CFFF796FD83
:100B800002E0002301976B62FFF7E4FB00980199F4
:100B900003F0FEFB6B6A002B01D0FFF733FC084B20
:100BA00094331B68002B03D100F046FB01242BE794
:100BB00004F058F927E7C04620BF0200580C001087
:100BC000BC0400100CFEFFFF8C0200103D52000020
:100BD00048010010080000103C0100100000001047
:100BE00014010010F0F1FFFF73B501F0F9FF3A4C6A
:100BF00000F0BAFC3948002101F074F900213848AE
:100C000001F070F900F088FD00F028FF2368072646
:100C1000B3432360236801252B4300202360021C7B
:100C20000B2101F0E9F8201C2E4C102101F05AF99B
:100C300023680022B34323602368281C2360042117
:100C400001F0DAF8201C002101F04CF901F0BEF8A7
:100C50009620000201F038FD234D01235B42002065
:100C60002B60FFF715FD00232B6050240120FFF7B8
:100C7000E9FA00F0F3FE02F0B1F82B68002B05D181
:100C80006420043C01F0EAFA142CEFD10020FFF7B5
:100C9000FFFC164801F000FF192001F0DFFA01F017
:100CA000B7FD002802D0FFF7BFFB02E0013C002C9B
:100CB000F2DC02F0EFFA03F0ABF91E2300930F23EE
:100CC00001930B480B490C4A0C4B03F0B3F90C4849
:100CD00003F0E2F9FFF790FE7440044098400440AE
:100CE0009C400440944004404801001047520000DA
:100CF000E14E000001030000650600008C020010B8
:100D000078020010F7B500283BD00378303B5A42F8
:100D10005341C0180378782B03D1013010260125E8
:100D200001E00A2600250378002201922D2B02D132
:100D300001230130019300230278002A1BD0171CE5
:100D4000303FFCB2092C02D87343DB1911E0202795
:100D50003A43002D08D0171C613FFFB2052F03D87E
:100D60001B01573A134304E0064801F095FE0020AA
:100D700007E00130E0E7019A002A00D05B420B60F7
:100D80000120FEBD515200000378202B01D101301B
:100D9000FAE77047031C303BDAB2092A01D8181C65
:100DA0000AE020231843031C613BDBB2052B01D86A
:100DB000573801E001204042704770B50E1CFFF724
:100DC000E3FF0025041C2078002807D0FFF7E2FF8E
:100DD000002803DB2D0105430134F4E73560201CB6
:100DE00070BD000008B500F023FD011C014801F0B2
:100DF00053FE08BD5F52000000B589B0684602F09E
:100E00008DF86946024801F047FE09B000BDC046B2
:100E10009B520000F7B50F1C01A9161CFFF772FFCB
:100E2000002814D0019C0B49201C04F059F90D1C1A
:100E3000081C642104F054F9281C3970642104F062
:100E4000F9F804493070201C04F0F4F801E00120A6
:100E50004042FEBD1027000037B50D1C48686A46A9
:100E6000694607310632FFF7D5FF01AC69466A468D
:100E700020800132A8680231FFF7CCFF6B46187062
:100E80002288044B9A4203D9201C694602F0D5F807
:100E900037BDC0466B07000007B5486801A9FFF7DA
:100EA00031FF019B3C20584302F0E0F807BD0000F1
:100EB00007235843054A10189C30013B04D3C25CF9
:100EC000002AFAD0002000E001207047BC04001086
:100ED00030B5194885B001F0DFFD0024651CA3077B
:100EE00019D1201CFFF7E4FF002810D0281CFFF7C1
:100EF000DFFF00280BD0A01CFFF7DAFF002806D088
:100F0000E01CFFF7D5FF002801D004340EE00B48A9
:100F1000211C01F0C1FD211C684602F0CFF9684692
:100F200001F078FE064801F0B7FD2C1CFF2CD5DD42
:100F300001F07EFE05B030BD645100006B52000030
:100F40005D9A000070B50E1CFFF71EFF0D25041CF6
:100F50000134631E1878FFF71DFF002806DB70556B
:100F6000013DF5D2201CFFF70FFF00E0002070BD0F
:100F700070B5444C86B023680868251C002B06D148
:100F8000414801F089FD03F043F8012309E0012BFA
:100F90000DD13E49082201F0EEFD002803D123685F
:100FA000013323606BE03A4801F076FD5FE003789F
:100FB000412B17D1374C0230211CFFF7C3FF00280B
:100FC00055D00378422B52D1211C02300E31FFF74D
:100FD000B9FF00284BD00378432B48D1211C0230A5
:100FE0001C3103E0532B06D12B490230FFF7AAFF37
:100FF000002844D13BE04D2B1FD1284C0230211C4E
:10100000FFF7A0FF002832D003784E2B2FD1211CF0
:1010100002300E31FFF796FF002828D00378472BC7
:1010200025D1023001A9FFF7C8FE019B002B1EDB72
:10103000184A1B4853651B491DE001A9FFF7BDFE77
:1010400004782023061C9C4311D1301C02A9FFF711
:1010500079FF019B061CE118FF2902DC02A802F0BF
:1010600043F9002E03D00134042CEED107E002F046
:10107000CFFF0B480C4901F00FFD00232B6006B099
:1010800070BDC0464C020010745200006451000054
:101090008A520000BC04001002050010E604001093
:1010A00096520000C1510000A052000037B54C68B4
:1010B0002378002B25D0201CFFF766FE01A9FFF73F
:1010C0007CFE019B041C002B1BD0D8B2FF2B09DD3A
:1010D00000F022FA019B051C1812C0B200F01CFAA5
:1010E000019003E000F018FA002501900198002813
:1010F00002D0291CFFF768F923785A1E9341E4189F
:10110000D6E737BD064A08B5137801214B40137066
:1011100001D0044900E00449044801F0BDFC08BDC9
:101120007003001044520000A7520000AB520000B0
:1011300007B5486801A9FFF7E5FD019B002B01DC1D
:1011400001230193019B1E2B01DD1E2301930199B5
:10115000034A044B4A4304481A6001F09DFC07BD52
:10116000701700006C030010BA52000038B5051C5F
:10117000002D09D0642402200021013C00F062FE11
:10118000002CF8D1013DF3E738BD70B5061C0120F5
:101190000821021C00F080FE072401200821002203
:1011A00000F07AFE321C012522412A400020022153
:1011B00000F072FE281C08212A1C00F06DFE013C84
:1011C000EBD270BD10B50021041C0A1C022000F0F7
:1011D00063FE201CFFF7D9FF10BDF0B5012385B0D9
:1011E00002930023061C039372B6002402AB1B5922
:1011F000502040421843C0B2FFF7E4FF0020FFF741
:10120000E1FF1020FFF7DEFFE020FFF7DBFF2127E3
:1012100067430025F71902200021012200F03CFE5F
:10122000785D0135FFF7B1FF842DF4D10434082C2B
:10123000DCD162B605B0F0BD08B5AC20FFF7C2FF47
:10124000AE20FFF7BFFFA520FFF7BCFF08BD38B5F4
:101250000122051C0C1C00F0CFFD281C211C0122C2
:1012600000F01AFE38BD08B5AF20FFF7ABFFA42091
:10127000FFF7A8FF08BD08B5AE20FFF7A3FF08BD24
:1012800010B5041CF820FFF79DFF201CFFF79AFF04
:1012900010BD10B5041C8120FFF794FF3F202040B3
:1012A000FFF790FF10BD000008B5074B20201B780A
:1012B0001843FFF787FF0A20FFF758FF034B187802
:1012C000FFF7E7FF08BDC046000000103C0100101A
:1012D00008B5842202480021520001F017FC08BD25
:1012E0007103001008B50248FFF777FF08BDC0463C
:1012F0007103001008B501200821FFF7A8FF0020A6
:101300000221FFF7A4FF02200021FFF7A0FF022027
:101310000621FFF79CFF0320011CFFF798FF032025
:10132000011C002200F0B8FD02200621002200F07E
:10133000B3FD06210122022000F0AEFDFFF7C8FF39
:10134000FFF7D0FFA220FFF73DFFA020FFF73AFFF5
:10135000C020FFF737FF0020FFF792FF0A20FFF7BA
:1013600005FF4020FFF72EFF2C20FFF72BFF322038
:10137000FFF7FCFE2E20FFF725FF3220FFF7F6FED9
:101380002F20FFF71FFF0A20FFF7F0FEFFF78CFF6B
:10139000FFF769FF08BD000083280ED80F290CD87D
:1013A000CB08842253430722C0181140034B8022EC
:1013B0000A41111C1A5C1143195470477103001043
:1013C000F7B55B18DBB20193019B994215D28425D6
:1013D000CC086C4307270F40802504193D41EFB22C
:1013E000A618B44206DA054D65192B7801343B4343
:1013F0002B70F6E70131C9B2E6E7F7BD71030010C3
:10140000F0B51E1C87B00592F27804915B688242A9
:1014100001D2307845E0244AB478934205D10322C2
:10142000041B54430192E4180CE0001B002282428A
:1014300004DA1978013202315B18F8E71A789C1C3B
:101440005B780193A218002503922F1C019B9F42F9
:1014500026DA08220023029200937378009A9A42B7
:101460001CDA029A082A06D1039B9C4218D000225B
:10147000257802920134EB0708D5049A009BB8182E
:10148000059AC0B29918C9B2FFF786FF009B029A6D
:10149000013301326D1000930292DEE70137D5E788
:1014A000019807B0F0BDC046DE520000F7B5041C3D
:1014B0000D1C161C1F1C01F04CFB20180190019BF9
:1014C0009C420BD0832D09D82078291C321C3B1C50
:1014D000FFF796FF01302D180134F0E7F7BD00004B
:1014E00010B50021012204230A4C0C5D844203D173
:1014F00018010243D0B20BE0013B002B04D10132B2
:10150000092A00DD1A1C042301312829ECD100200E
:1015100010BDC046A45A00000F23020918408000E5
:10152000031F00D52833511E0020032906D8242B81
:1015300004DC04218A1A0249CB18985C7047C04623
:10154000A45A000038B5051C0024054B291CE05C9A
:10155000044B0134C01800F0C5FC0A2CF5D138BD8D
:10156000E05A000000400440F8B50D4F3C68002CE4
:1015700015D11020FFF7E6FF0A4B0022E65C1B198D
:101580005D78301C291C00F037FC0234301C291C0B
:10159000012200F081FC142CEED101233B60F8BD48
:1015A00040010010CC5A000070B500240B4B012202
:1015B000E65C1B195D78301C291C00F01DFC023410
:1015C000301C291C002200F067FC142CEED10020F6
:1015D000FFF7B8FF024B00221A6070BDCC5A000022
:1015E0004001001038B5051CFFF7BEFF002D09D0E3
:1015F00007210122022000F0FFFB104B80211A6816
:101600008A431A6000200B2100F01CFC01240028F2
:1016100005D000200B2100F015FC44424441002D70
:1016200009D007210022022000F0E6FB034B8021B5
:101630001A680A431A60201C38BDC046FC3F02509D
:10164000F0B587B00026029001200391049605961C
:10165000FFF7C8FFB04202D01823049301260021EF
:10166000284C009120786178012200F0C5FB207899
:101670006178002200F010FC234B9D1D012E24DC1C
:101680006A782F78111C381C019200F0DBFB0028CF
:1016900008D100991D4AB3008A5C103369465A503C
:1016A00001360BE02878697800F0CCFB0028F0D0F8
:1016B000381C019900F0C6FB0028EAD0009A144BB0
:1016C0000132023D00929D42D8D127786578381CBE
:1016D000291C002200F090FB291C381C012200F07C
:1016E000DBFB0C4902348C42BCD10020864206D080
:1016F000049A029B05991A60039A0120116007B0B1
:10170000F0BDC046CC5A00009C5A0000A45A00000C
:101710009A5A0000E05A000008B50120021C0B2173
:1017200000F06AFB01200B21002200F0B5FB032032
:101730000221012200F060FB03200221002200F0C0
:10174000ABFB08BD234B37B51A6810218A431A60DA
:10175000214B8022196892010A431A60051C0B2153
:101760000120002200F048FB01200B21002200F0A4
:1017700093FB1A4B9F211A68194C8A431A601A6806
:1017800018491A60184B186803F054FC80230002B3
:1017900018432A1C20600221032000F07DFB142046
:1017A00000F05CFD2368FF229343236023680F4A07
:1017B000134323600E4B1B680193019B002BF9DA46
:1017C00022680C4B13402360FFF7A6FF019800042A
:1017D000800D3EBD38820440808004409840044023
:1017E00000C0014000093D0080040010800000019D
:1017F0002CC00140FFFFFFF810B50C4C20680028FA
:1018000013DA00202060FFF79DFF0A280ADC012080
:10181000FFF798FF0138C023FF385B00984201D8DA
:1018200001232360FFF778FF206810BD040000103B
:1018300008B5FFF7E1FF002801D1002007E00120F3
:10184000FFF780FF011EF8D0014803F0F3FB08BD4D
:1018500050BB120008B5FFF7CFFF00280AD0FFF7F2
:10186000E7FFFA22031C0021C00FD2009A42484130
:10187000014B186008BDC0464401001008B5074B75
:1018800002221A60064BA2221960064B1A70A3228C
:1018900058709A7000F0F2FD08BDC046AC0400100C
:1018A000880400109C04001008B5064B0231196032
:1018B000054B00221A60054BA2221A70587000F0E6
:1018C000DDFD08BDAC040010880400109C0400106D
:1018D00070B5051C0E1C0324281C311CFFF7CEFF1D
:1018E0000223FF33984202D0013C002CF4D170BD9A
:1018F00070B5051C0E1C0324281C311CFFF7D4FFF7
:101900000223FF33984202D0013C002CF4D170BD79
:101910000B4B10B51C6800239C420ED0094CA31C35
:10192000A270140A5C70140C120EDA709C70FFF72F
:10193000DFFF831EFF3B5A425341181C10BDC046B7
:10194000480100109C04001070B50E4C256800245E
:10195000A54215D00C4C160AA270E670160C120E99
:101960006271A371A21D26711C0A54701C0C1B0EFF
:101970009470D370FFF7BCFF841EFF3C63425C4150
:10198000201C70BD480100109C04001008B5064BD7
:101990001A6800239A4205D0FFF79AFF831EFF3B87
:1019A0005A425341181C08BD4801001008B5074BA6
:1019B00000201B68834207D002200721FFF788FF21
:1019C0000238FF384342584108BDC0464801001064
:1019D00038B50F4B051C1B680020834217D0092423
:1019E000641B631E062B10D8072C05D00948A91EBE
:1019F0000918221C01F068F8E8B2211CFFF778FFF3
:101A00000238FF384342584101E00120404238BDCE
:101A1000480100109E040010012010B5011CFFF7C2
:101A200057FF0223FF3398420ED1094B0121196061
:101A3000084B1C78230709D0074B032222409A70D9
:101A4000081CFFF755FF01E001246442201C10BD73
:101A5000480100108C0400109C04001008B5FFF72A
:101A6000DBFF02200121FFF733FF0223FF339842FF
:101A70000FD1084B1B787F2B06D984220220072127
:101A80005204054BFFF760FF09200421034AFFF7CA
:101A90003FFF08BD8C04001002011400808080808C
:101AA00010B500280CD0254B80211A688A431A6093
:101AB000234B1B68D907FBD5224B03221A6001E098
:101AC000204B1860204B012200211A6019601A6017
:101AD000196801221142FBD01C4B80211A601C4A5C
:101AE00049021468214311601A1C002804D1134BC9
:101AF0008024196821431960164B196888421CD04C
:101B00001860002801D0144800E01448116803F060
:101B100043FA134BFA2118608900041C03F08AFA77
:101B20001E2358430F4BC82118604901201C03F0A5
:101B300081FA0D4B186001F03DF810BD3882044069
:101B40000C8004407080044074800440788004401D
:101B50008080044008000010006CDC02001BB7000D
:101B6000800400107C0400108404001008B500F00C
:101B700035F9134B00211A68120B12031A60114B2E
:101B80001A68120B12031A600F4B1A68120B120319
:101B90001A600E4B1A68120B12031A600C4B0122CA
:101BA00019600C4B1A6019601A601A680120024211
:101BB000FBD0094B23221A60FFF772FF08BDC04615
:101BC00000800050008001500080025000800350CF
:101BD00040800440448004400880044038B50F49E8
:101BE0000F4800F059FF0F4D0024281C00F054FF4F
:101BF0000D4A0E48A1581219D2682B1C143400F05B
:101C00004BFFC82CF4D10A4800F046FF00F046FB19
:101C1000011C084800F040FF38BDC0466451000078
:101C2000EA5A00003A5B0000305C0000FC5A0000F9
:101C3000075B0000295B0000F0B53B4B8BB01E68D2
:101C4000041C002E01D1351C08E0384B02901B68A3
:101C500001209B6854E033681E79019D2378002B96
:101C600031D0082D33D02378202B01D10134FAE76D
:101C7000002B28D06A1CAD0008356B460192EC5051
:101C8000FF2E4CD02278002A07D0631C202A01D0D6
:101C90001C1CF7E7002222701C1C019A012ADCD1CF
:101CA000224E234B0B253360371C013D002D2ED0D7
:101CB0003B680298196800F06FFF0028CBD03B68A2
:101CC00014333B60F1E7002D1CD0022D02D0B54249
:101CD00006D911E00398174900F05EFF0028F6D1FD
:101CE000124C15482368D96800F0D6FE23681348C3
:101CF000196900F0D1FE05E00C4BE8B21B689B6847
:101D000002A99847084A1368002B0BD103E0281C4E
:101D1000291CFFF763FF0A4800F0BEFE02E0019DA8
:101D20000026D2E70BB0F0BD4C02001054020010A8
:101D3000305C000091510000365B00009B520000B7
:101D40003D5B000038B5041C164D0A2808D002D8A7
:101D5000082811D01CE00D2802D07F280CD017E0F5
:101D60002A6800231370104800F096FE0F4C201CC8
:101D7000FFF762FF2C6013E00C4B2A689A420FD9E0
:101D80000B48211C00F088FE2B68013B2B6007E00C
:101D90000748211C00F080FE2B685A1C2A601C702A
:101DA00038BDC046500200103A5B00004C010010E4
:101DB000495B000008B500F02BFD002804D000F0BE
:101DC000FDFCFFF7BFFFF6E708BD0000014A024B2C
:101DD0001A6070474C01001050020010044B402163
:101DE0001A680A431A60034B01221A707047C046F2
:101DF00080800440580200100F4B70B51B78061C01
:101E00000C1C151C002B01D1FFF7E8FF701E0228E7
:101E100003D80A4B8000C35800E0094B1A68012D13
:101E200004D1A5402C1C14431C6003E00121A140F7
:101E30008A431A6070BDC04658020010F85C00006A
:101E40000080005038B50F4B051C1B780C1C002B74
:101E500001D1FFF7C3FF0020032D12D8281C012257
:101E600003F086F802040608074B04E0074B02E083
:101E7000074B00E0074B1B68A2401340181C421E92
:101E8000904138BD58020010FC3F0050FC3F01500B
:101E9000FC3F0250FC3F03500F4B70B51B78061CF3
:101EA0000C1C151C002B01D1FFF798FF701E022897
:101EB00003D80A4B8000C35800E0094B1A68012D73
:101EC00004D1A5402C1C14431C6003E00121A14057
:101ED0008A431A6070BDC04658020010045D0000BD
:101EE000FC3F005038B5084B041C1B780D1C002B20
:101EF00001D1FFF773FF23681822934323602368FF
:101F00001D43256038BDC04658020010054B3F22D6
:101F10001A60054B01221A60044B40211A688A435B
:101F20001A60704724800440D880044038820440FE
:101F300008B5044B40211A688A431A60FFF7E6FF90
:101F400008BDC0463882044008B500F05DFAFFF7CE
:101F50002BFB0A480021FFF7C5FF09480021FFF7C6
:101F6000C1FF08480021FFF7BDFF07480021FFF728
:101F7000B9FF06480021FFF7B5FF08BD084004403F
:101F800000400440AC400440144004401C40044065
:101F900008B50120FEF756F908BD000008B5124B40
:101FA0008022DA675200DA678022D200DA67802264
:101FB0005201DA6780221201DA6780229200DA6722
:101FC0000A4A002313600121094A49421160094A63
:101FD0001360094A1360094A01231360084A136019
:101FE000FFF7D6FF08BDC04604E100E004820440CC
:101FF0000882044004C000403CC0004000C00040D3
:102000000040014008B5064B1A6801321A60054BC2
:102010001868FFF745FDFFF7C1FFC046C04608BD81
:102020005C02001008000010F7B5071C0C1C72B60B
:10203000FFF78AFF524B1A68524B1A60002F01D0EB
:10204000514B00E0514B524A04211360514B524D09
:102050001A680A431A6000232B60A1071ED04F4B59
:102060004F4A19680A401A6029684E4BA2070ED5DC
:10207000EC2252010A432A6080221A6052001A6040
:102080008022D2001A60802252011A6003E080226E
:1020900012010A432A60802212011A60002F53D0D5
:1020A000414B00241C60414B414E1C60414B301C95
:1020B0001C60414B211C1C60FFF714FF201C0921F0
:1020C000221CFFF799FE201C0921221CFFF7E4FEC9
:1020D0003A4B80211A683A480A431A60336807224B
:1020E0009343336033680222134333600A217843F9
:1020F00002F052FF334B03221860334B1C60334B0A
:102100001A60334B334A19680A401A601A688021F2
:102110000A431A60234A8B001360204A116819434E
:1021200011602A68022113432B602B4B01221A6095
:102130002A4B19602A4B1C491A601C601A601868E7
:1021400001221042FBD00A60264B012252421A6043
:10215000254B00221B680193244B1A6062B630BFE6
:10216000C046214B019A1B689A4208D11F4B01229D
:102170001A601F4B1868FFF793FCFFF70FFFF7BDBE
:102180003882044034820440BF180000FF18000069
:102190003082044010ED00E00482044000820440DC
:1021A0007FE2FFFF00E100E004C0004004000140C6
:1021B00064400440044001400480014080800440A9
:1021C000841E000018C0004008C0004014C0004039
:1021D0003CC000400FF0FFFF788004407080044056
:1021E00074800440088204405C0200106002001009
:1021F0000800001008B5FFF717FF08BD074B1A6865
:10220000013203D1064A1168013111601A680132A6
:102210001A60044B1A6801321A607047700200108D
:102220006C02001064020010074B98420AD8074A5B
:1022300000231360064A01381060064A1360064BFB
:1022400007221A607047C046FFFFFF0070020010AF
:1022500014E000E018E000E010E000E00B4A10B5E8
:102260001368002800D10120C1438B4208D91168AE
:10227000994209D3591C146809188C42FAD3F6E71D
:102280001168C91A8142FBD310BDC046700200100C
:10229000014B18687047C04670020010064BFA21C7
:1022A0001868064B10B589001C6802F075FE044BD7
:1022B0005C43201810BDC046700200106C02001074
:1022C00037894100034B01221A60034B1A6801321F
:1022D0001A60704700C0004074020010034B0122D6
:1022E0001A60034B1A6801321A60704700000140FF
:1022F00078020010002803D1044B01221A6003E089
:10230000012801D1024B18607047C04604C000404C
:1023100004000140002802D1044B186004E00128A9
:1023200002D1034B00221A607047C04604C000402F
:1023300004000140002801D1044B02E0012804D12F
:10234000034B1A6802210A431A60704704C0004018
:102350000400014010B5002900D1134900280DD117
:10236000124B80241A6822431A60114B0322186012
:10237000104B1960104B1A60620211E0012811D154
:102380000A4B80221868520002431A600B4B00224D
:102390001A600B4B032219600A4B1A6080229202CA
:1023A000094B1A6010BDC046FFFF0000808004404A
:1023B0007402001018C0004014C0004078020010E1
:1023C000180001401400014000E100E080231022C9
:1023D000DB051A60094B08221A6000238022D2050F
:1023E0001268D10604D5064A934201D00133F5E7BD
:1023F000044898429B4158427047C046180000402C
:10240000FF0F0000FE0F000008B58022154B1202DE
:10241000DA67154B6C221A60144B154A19680020B4
:102420001140196019681960124B19680A401A6046
:102430001A6804211A600122FFF7DEFC0020042143
:102440000122FFF729FD002005210122FFF7D4FC1E
:10245000012200200521FFF71FFD074B00221A6013
:1024600008BDC04604E100E01800004030400440D0
:10247000F8FCFFFF3440044004800440F8B5174ADC
:10248000174C002323601360164A2021136080221A
:10249000D20511602168144A012903D0934203D068
:1024A0000133F7E7934203D1FFF790FF002014E0D8
:1024B0000E4F00253E68013E2368FF2B0CD83B6879
:1024C0009E4204D03E68FFF7E3FE051C0A35FFF785
:1024D000DFFE8542F0D1E7E72068F8BD7C020010FE
:1024E0008002001084020010FF0F0000880200101C
:1024F000034B01221A60034B1A6801321A607047BD
:10250000004001408C020010174B70B501241C6084
:10251000164B1A6812191A60154B1A68002A22D035
:102520001A68144D013A1A601E68002E0DD02A68F0
:10253000201C211CFFF7B0FC2B68201CE31A2B6029
:102540002A680221FFF7A8FC0DE01B68201C2B6005
:102550002A68211CFFF7A0FC2A68201C0221FFF733
:102560009BFC054B1E6070BD008001409402001072
:10257000900200109802001004800140002803D14E
:10258000044B01221A6003E0012801D1024B1860BC
:102590007047C0460440014004800140002802D139
:1025A000044B186004E0012802D1034B00221A609A
:1025B0007047C0460440014004800140002801D11A
:1025C000044B02E0012804D1034B1A6802210A439C
:1025D0001A607047044001400480014010B5002893
:1025E0000FD1124B80221C68920022431A60104BBC
:1025F000032218600F4B19600F4B1A608022D20221
:1026000011E0012811D1094B80221868D200024341
:102610001A600A4B00221A60094B03221960094B09
:102620001A6080221203084B1A6010BD808004409B
:102630008C02001018400140144001409402001028
:10264000188001401480014000E100E008B5184BFB
:102650001A680E231340062B0DD1164B9E221B68C1
:10266000134205D0144ADBB25360144B1B681EE0C2
:10267000D9071CD501E0042B05D1104B1868C0B256
:1026800000F0B1F813E00C2B06D10B4B80225968F7
:1026900052000A435A600AE0022B08D1054B1A681F
:1026A000054B910601D5002200E001229A6008BD89
:1026B00008800040148000409C0200100080004010
:1026C000004870479C020010F7B52D4B2D4C80221E
:1026D000002192030191061CDA67201C902200F071
:1026E00015FA019B0725A360274B284F1A68AA43B8
:1026F0001A601968012211431960254B1968A94312
:102700001960196811431960224B8021186849012A
:1027100001431960204B1A6083223A601F4A1268F5
:1027200019681F4B1868504302F036FC311C000931
:1027300002F032FC1B4B10221B491A60030A0B608B
:102740001A4BC0B2032218603A60194A1560194A40
:102750001D1C10680190106860230340602BFAD1A3
:1027600010680123184202D02B680193F8E7237008
:102770008022114B92031A6005230B60F7BDC046FF
:1027800004E100E09C020010A44004400C800040E2
:10279000A840044080800440988004407880044031
:1027A0008004001028800040048000400080004029
:1027B000088000401480004000E100E008B5FFF709
:1027C0007FFFC268031C1202120E8218D07BDA68E7
:1027D0001202120E0132D2B29A7352B2002A01DAF8
:1027E00000229A7308BD10B5041CFFF769FFC26888
:1027F0001204120E8218D473C2681204120E01322F
:10280000D2B2427352B2002A01DA0022427310BDE2
:1028100008B5FFF755FFC268C36812021B041B0E00
:10282000120ED01A431E9841C0B208BD70B50024E4
:102830001D5D0619002D02D005550134F8E7121B65
:10284000301C131C002B03DD0170013B0130F9E744
:10285000D043C0170240A01870BDF7B5051C019108
:102860000093561E092B01D8041C0CE000980A2185
:1028700002F092FB0199031C321C281CFFF7EDFFAC
:10288000071C2C1807E0671B002E04DD019B013E8E
:1028900023700134F7E700980A2102F0C1FB3031C0
:1028A000781C2170FEBDF8B50C1CD9175F18051CEB
:1028B0004F40561E092F12D9381C0A21002B03DA6B
:1028C00002F06AFB434202E002F066FB031C281C94
:1028D000211C321CFFF7E7FF041C2D1814E0002B0D
:1028E00000DA961E2A1CA919891A002902DD147023
:1028F0000132F8E7F443E41734402D19002B03DAD2
:102900002D232B7001340135381C0A2102F088FB7D
:1029100030312970601CF8BDF7B5089F1E1C051CDE
:10292000013A3B0901D1041C05E00093331CFFF779
:10293000F3FF2C1806E0601B002A03DD2170013A2A
:102940000134F8E70F231F40092F01D8303704E086
:10295000002E01D0373700E0573727700130FEBD19
:10296000F0B585B0041C029101D000210170002552
:102970001178002906D1029F0023BD426CD223703A
:10298000281C6FE0029FBD42F5D2252902D00132FA
:10299000217004E05178252904D1217002320135DB
:1029A0000134E5E7302902D0561C202100E0961CB6
:1029B00032782D3A50424241B61800223078302702
:1029C0007F423F18FFB2092F07D80A277A4382189F
:1029D000D2B2303AD2B20136F0E7AF18BC46029F0D
:1029E000BC4501D97A1BD2B2692818D00BD863280C
:1029F0002AD0642813D0582832D11F1D1B68201CF0
:102A0000009301231DE075280FD0782814D0732877
:102A100026D11F1D201C1B68FFF708FF0AE01F1DA1
:102A2000201C1B68FFF73FFF04E01F1D201C1B68D4
:102A3000FFF713FF3B1C0BE01F1D1B68201C0093BE
:102A40000023FFF769FFF5E71868043320700120C1
:102A5000721C24182D188BE7013C2370681E01E0BE
:102A60000120404205B0F0BD10B50C1C131C6421C0
:102A7000221CFFF775FF10BD00B5031C9BB00A1C9C
:102A800001A8191CFFF7F0FF632800DDFEE701A88D
:102A900000F0B6F81BB000BD0FB407B504A908C913
:102AA000181C0191FFF7E8FF03B008BC04B01847F9
:102AB0000EB403B503AA08CA191C0192FFF7D4FF8C
:102AC00002B008BC03B0184730B50C1C0443032304
:102AD0002340041C002B01D0002310E0032AFBD963
:102AE000CC58C4500433D41A032CF9D8131F9B08B4
:102AF00001339B00C418C91803231A40ECE7934222
:102B000003D0CD5CE5540133F9E730BD30B5031C8B
:102B1000840701D1032A01D89A1814E00B060C048B
:102B20001D1C25430D430C022543031C20C38418A0
:102B3000E41A032CFAD8131F9B0801339B000324CB
:102B4000C3182240E8E7934202D019700133FAE734
:102B500030BD021C031C981A0133591E0978002944
:102B6000F9D17047031C0A781A70002A02D001318B
:102B70000133F8E7704730B50023934208D0C45CB6
:102B8000CD5C651B06D10133002CF6D1201C02E080
:102B9000002000E0281C30BD10B50022835C8C5C56
:102BA000A34204D10132002BF8D1181C00E0181BFD
:102BB00010BD000008B5094BFA211868890002F021
:102BC00039FAFFF731FB96200002FFF77DFD012067
:102BD000FDF738FBFEF742FF08BDC0468004001039
:102BE00008B5FEF7C3FFFFF7F9F8FFF7A1F9FEF705
:102BF00081FBFEF76DFBFFF7DDFFFFF7E7F808BD90
:102C000010B5041C2078002803D00134FDF76AFBBE
:102C1000F8E710BD38B5051C0E24013C04D3295D2E
:102C20000248FFF739FFF8E738BDC046105D0000E5
:102C300038B51948FFF730FF184C201CFFF7EAFFA2
:102C4000174D4221281CFFF727FF201C0E30FFF7ED
:102C5000E1FF4321281CFFF71FFF201C1C30FFF75A
:102C6000D9FF1048FFF718FF201C4630FFF7D2FFAE
:102C70000D48FFF711FF201C2A30FFF7CBFF281C5F
:102C80004E21FFF709FF201C3830FFF7C3FF616DAD
:102C90000648FFF701FF38BD135D0000BC040010BB
:102CA000195D0000205D0000265D00002C5D000025
:102CB00003110A2253430F2210401818704738B5E9
:102CC0000A21041C02F0B6F90A210501201C02F0B9
:102CD00007FA281C084338BD08B5C12252000E204F
:102CE0000221FEF715FE024B01225A7108BDC046B3
:102CF000B004001010B5084C6379002B01D1FFF728
:102D0000EBFF23790C221A43A37901205B001A43BD
:102D1000011CFEF7FDFD10BDB004001010B5074CFE
:102D20002379002B08D16379002B01D1FFF7D4FF61
:102D300001232371FFF7DEFF10BDC046B004001071
:102D400008B5054B1A79002A05D000221A711A72AB
:102D5000DA70FFF7CFFF08BDB004001010B50121F5
:102D60000220FEF713FE064B041C18787F23184040
:102D7000FFF79EFF034B5870DC71201C10BDC0464E
:102D80008C040010B0040010014B01229A707047AF
:102D9000B0040010024B00229A701A727047C046AD
:102DA000B004001008B5FFF7D9FF094B094A99781C
:102DB000002908D0197A012901D8013103E01068EF
:102DC0000549086000E019720021D970116008BD42
:102DD000B0040010640200106802001008B5FEF78D
:102DE0001BFE0C23184003D0024B1A7810431870B6
:102DF00008BDC046B004001010B5FFF7EFFF054B4B
:102E00001A781C1C530701D5FFF7CCFF0023237051
:102E100010BDC046B004001008B50020FEF7E2FB6C
:102E2000002801D0FFF7E8FF08BD000010B5054CF1
:102E30000023E371FFF7F0FFE379002B01D1FFF7E7
:102E40008DFF10BDB004001008B50948092102F03B
:102E500053F9084BFA22D2001A80FFF7E7FF064B1E
:102E600000221A60FA22054B92001A6008BDC04683
:102E7000B0040010BA0400106402001068020010D0
:102E800008B5FFF7C9FF002008BD08B5FFF758FFD8
:102E900008BD000070B51D4C061C637822781B022B
:102EA0001343A278A07912041343E2780D1C120692
:102EB0001343174A13401A0A237062701A0C1B0E30
:102EC000E3706379A27022791B021343114A134005
:102ED00023711B0A6371FFF7EBFE0F4B1B88C018B1
:102EE00030806079FFF7E4FEB070E078FFF7E0FE35
:102EF000F070A078FFF7DCFE28706078FFF7D8FE4E
:102F000068702078FFF7D4FEA87070BD8C040010A4
:102F10007F7F3F3F071F0000BA040010F0B58DB05F
:102F2000051CFEF743FD002804D1281C1249FFF7B9
:102F3000BFFD1EE00AAE0BAC211C301CFFF7AAFF40
:102F40003388F7780793B378267808936378A47862
:102F500009930A4B187900F0D7F8099B0490029363
:102F6000009701960394281C0549079A089BFFF7D0
:102F70009FFD0DB0F0BDC046385D00008C04001010
:102F80003D5D000070B5061C0D1C141CFEF70EFD07
:102F900000280AD0301C291CFFF77CFF002C07D02A
:102FA000044B00201B79236003E00120404200E035
:102FB000201C70BD8C040010F7B504880E1C051C85
:102FC0006421201C0092019302F02AF8114B8FB269
:102FD000B078E41B1C80FFF772FE0F4CA070707875
:102FE000FFF76DFEE0703078FFF769FE2071E8783A
:102FF000FFF765FE009B6071A371A878FFF75FFE85
:10300000E071381CFFF75BFE20720198FEF7E0FCD0
:10301000FEBDC046BA0400109C04001008B502238F
:10302000FFF7CAFF08BD08B5021C501E82415201BD
:1030300000200121FEF76CFC08BD38B5041C0120FE
:103040000D1CFFF7F0FF201C00F086F8072102F0AE
:1030500047F8201C0A1C291CFFF7E0FF96204000BF
:10306000FFF7FCF80020FFF7DEFF38BD73B5041C46
:10307000FFF774FE002801D100203BE01E4B5D7875
:103080001E1C7378AB4207D10A20FFF7E7F8FFF761
:1030900065FE0028F5D1EFE7FEF788FC0028EBD0AD
:1030A00001A96846FFF7F6FE684600F055F8051CD2
:1030B00001A800F031F8114B04199C420DD9E31717
:1030C00001221343ED18281C694600F075F8002C06
:1030D00001DA0B4B00E00B4BE418201C01A900F0B7
:1030E00024F8281C072101F0FBFF68460A1C01A9EF
:1030F000FFF794FF76BDC046B00400107F51010079
:103100008051010080AEFEFF07231840014B800074
:10311000C0587047B05D000002783C235A434178A4
:103120005218534382789818704738B50C1C3C21CC
:10313000051C01F0D5FF281CA1703C2101F07AFF8D
:103140003C2101F0CDFF6170E121281C090101F053
:1031500071FF207038BD000070B583780221002215
:1031600099425241048896214901051C64180C209B
:10317000A41A42439B18033B99205843052102306F
:1031800001F058FF6E26FF3666436421A3108619AE
:103190004942201CF61801F04DFFC821361849009D
:1031A000201C01F047FF034B3018C018EB78C01803
:1031B00070BDC046D382FFFFF8B5204B0C1CC5186C
:1031C0001F4B8000C0181F4901F034FF03235843F0
:1031D000C617B60F3618B610AE19B600953E301C9D
:1031E000194901F07DFFCD17AD0F6D180527AD1002
:1031F0007D430235281C992101F072FF081C391CFF
:1032000001F018FF0130E0709921281C01F012FF35
:103210000C21023001F064FF4D1CEDB2A570301C92
:10322000094901F007FF094B0C21C6180E20401B6D
:1032300001F000FF36182680F8BDC0467905000071
:10324000652F0400B13A0200B505000094EDFFFFC0
:10325000F8238A01DB0013404A05920E1343F8223B
:103260001202114019430A23594330B5CA1083187A
:103270001C1CEB345D782478EA336C401B78240204
:103280001C43835C201C58400723194008418005DB
:10329000800D30BD7047000008B5054B011E9942F6
:1032A00001DD044BC1180448EA38FFF7D1FF08BD1F
:1032B000FF17000000F8FFFFEC5D000007235943F3
:1032C00010B5084B59189C310023CC5C0F222240CA
:1032D0000270CA5C0133120942700230072BF4D12C
:1032E00010BDC046BC0400100723594310B5074B5E
:1032F00059189C3100234278047812012243CA54A1
:1033000001330230072BF6D110BDC046BC040010BB
:1033100070B5AD4C86B0E36E6E465A1E93411736BB
:103320003370AA4B9A6A191CD006400F0138062840
:1033300007D801F01DFE040C2012181A1D000225EA
:1033400009E0636E16339B001B591D1C15E0636E6C
:1033500016339B00E55800230FE0A36DE56DAB42EB
:103360000BDD0D2509E0022503E00C25032304E015
:103370000D252B1C01E00D25EDE70D6150111F28D7
:1033800000D91BE101F0FEFD2000220029002C00E5
:103390002F0033003B00440048004C005400610003
:1033A0006E00760083008F009B00A800B800C50067
:1033B000D500D300E100E400E700EF00FE000201C9
:1033C0000B010D010F011501E01801E0E0180E30AE
:1033D000EB1A591C01F090FEF0E0E0181C30F7E702
:1033E000211C0E3105E0E0180E30E1180BE0211C25
:1033F0001C31201C1A1C2B1C01F00BF9DEE0E0181C
:10340000E1181C300E31EB1A5A1CFFF75DFBD5E0BA
:103410006F48011C0E31EDE7E018011C1C31F2E78A
:10342000226E1021002A00D00A21221C0E3206E052
:10343000226E1021002A00D00A21221C1C32029187
:1034400000950196201C211C53E0216E0122327050
:103450001022002900D00A22009501960292201C19
:10346000211C45E0226E1021002A00D00A21221CD6
:103470000E3213E0216E012232701022002900D09A
:103480000A22009501960292201C211C4DE0226E1A
:103490001021002A00D00A21221C1C32009501961E
:1034A0000291201C6AE0226E1021002A00D00A211D
:1034B000484A029100950196101C111C19E0216EDA
:1034C0001020002900D00A20424A0290111C1C3909
:1034D00000950196101C0CE0216E01223270102222
:1034E000002900D00A223B49009501960292081C4F
:1034F000002201F098F861E0226E1020002A00D02E
:103500000A20344A0290111C1C3900950196101CA7
:1035100035E0216E012232701022002900D00A22EB
:103520002C49009501960292081C002227E00122F6
:103530003270226E1021002A00D00A21254A029101
:1035400000950196101C002119E0009620481BE010
:103550000096204818E0226E1021002A00D00A218F
:10356000221C1C3206E0226E1021002A00D00A2103
:10357000221C0E320095019602910020211C01F0C0
:103580007AF81BE00096201C002103E0211C1C316E
:103590000096201C1A1C2B1C01F0CAF80EE0201CFF
:1035A00002E00B4800E00B48191C2A1C01F0D7F878
:1035B00004E0201C191C2A1C01F0DBF833780120E0
:1035C000E36606B070BDC046BC040010580C001085
:1035D000CA040010D8040010064910B50A1C88322D
:1035E00013681C1C1E34A4006050013303210B40DF
:1035F000136010BDBC040010054B0322191C883158
:103600000868013802400A601E329200D0587047A4
:10361000BC040010F7B5124F3D1C8C3528680130F2
:10362000FFF73AFE0F4EBB6EB26A041C01920122F4
:10363000F06202409A4210D1830703D42868023016
:10364000FFF7CAFFFF239B00019A1C40A4019310BF
:103650001C438C3701233C60F3600220FEBDC04652
:10366000BC040010580C00100C490D488A6A031C59
:103670008C3370B51D68D3059B0E0C1C910500D5CD
:10368000403B866E921001210A40B24203D18C3039
:10369000EB180360E160012070BDC046580C0010BB
:1036A000BC04001008B5084B5A1CD07F9A1CD27F6E
:1036B00000011202104303331A7FDB7F10431B0308
:1036C0001843FFF789FF08BDBC04001008B5FFF7D9
:1036D00093FF0323044A0F219A1801400133117705
:1036E0000011072BF6D108BDBC04001008B5FFF788
:1036F00083FF034B01228C331860024BDA6008BD54
:10370000BC040010580C001010B5064CA36E002B22
:1037100006D0FFF771FF044B8C3401222060DA6081
:1037200010BDC046BC040010580C001010B5064C6B
:10373000A36E002B06D1FFF75FFF044B8C340122F0
:103740002060DA6010BDC046BC040010580C0010A8
:1037500008B5104B0022596A1A62914214D0596977
:10376000914216DD012906D1D969914203D0DA616F
:103770000A2299615A615A69032A02DD0649012029
:10378000C866013A5A6104E0044B1B68002B00D064
:10379000984708BD580C0010BC0400102C03001002
:1037A000074B5A6A002A02D05A69002A07DD9A6933
:1037B0000F21044B1140D97712110133DA7770478A
:1037C000580C0010BC040010044B597F9A7F09016B
:1037D00012020A43197F0A435A677047BC0400105B
:1037E0000B1C093B10B5012B0FD80023074A9A1870
:1037F000147FC25C944205D0054B08395A681143C6
:10380000596002E001330E2BF0D110BDBC04001052
:10381000580C001008B508290DD0192913D1427889
:1038200008231A4202D00022027002E00F23037024
:103830000723437005E000230022C25401330E2BFE
:10384000FAD1FFF751FD08BD30B5114D85B06C6F51
:10385000002802D00F239C4304436C67FF2C05DD36
:10386000281C1C300E2101F047FC0FE06846211C8B
:10387000FFF724FD6846211CFFF7CCFF00236846B4
:10388000C15CEA18013311770E2BF8D105B030BDB9
:10389000BC040010134B30B5596F0F229143041C28
:1038A0000C4385B05C671D1C082C19D0FF2C17DC5D
:1038B0006846211CFFF702FD6846211CFFF790FFB8
:1038C0000023EA18127F6946CA5401330E2BF8D13F
:1038D0006846211CFFF79EFF6846211CFFF704FD88
:1038E00005B030BDBC0400101FB50F4C616F082936
:1038F00018D0FF2916DC6846FFF7E0FC6846616FC8
:10390000FFF76EFF0023E218127F6946CA540133A5
:103910000E2BF8D16846616FFFF77CFF616F684638
:10392000FFF7E2FC1FBDC046BC04001010B50D4CF3
:10393000631CD87FA31CDB7F00011B021843E37FBD
:103940001843E31CDB7F1B031843FFF7A5FC0F2381
:10395000021C1A4022770211134000126377A077ED
:1039600010BDC046BC040010044B5A6E16329200C3
:10397000D258121A51424A41DA667047BC0400100C
:10398000044B5A6E16329200D158013900D50D21E0
:10399000D1507047BC040010054B5A6E163292008D
:1039A000D15801310E2900D10021D1507047C046B5
:1039B000BC040010094B5A6E16329200D2580D2AE0
:1039C00003D11A1C2932127805E09A18507F117F12
:1039D0000001021C0A435A657047C046BC0400102F
:1039E000084B10B55A6E0F2416329200D1585A6DFA
:1039F00058181440013104770D2902DC5B181211AC
:103A00001A7710BDBC0400100E4B30B55A6E596DBC
:103A100016329200D2580D2A07D11C1C2934F020EE
:103A2000247808402043586507E09818447F057FB4
:103A300024012C435C650C1144779B180F22114024
:103A4000197730BDBC04001008B503480E22011CD4
:103A50001C39FFF739F808BDF404001008B5034815
:103A60000E22011C1C31FFF72FF808BDD8040010EE
:103A700008B504480022011C1C310D2300F0C9FDCB
:103A800008BDC046D804001008B503480E22011C2A
:103A90000E39FFF719F808BDE604001008B5034811
:103AA0000E22011C0E31FFF70FF808BDD8040010DC
:103AB00008B504480022011C0E310D2300F0A9FDB9
:103AC00008BDC046D80400100023044A00219A18FB
:103AD000463201331170082BF7D17047BC04001037
:103AE000C31C421E0020934207D0044940005918CD
:103AF00046310978013B0843F5E77047BC040010E4
:103B000010B50B1D994208D0044A01248A180440BC
:103B10004632147040100131F4E710BDBC040010AF
:103B200038B50020FFF7DCFF084C051C0021207F82
:103B3000FFF7E6FF04202577FFF7D2FF0421051CDD
:103B4000607FFFF7DDFF657738BDC046BC0400101D
:103B500010B50020FFF7C4FF034C20770420FFF7C7
:103B6000BFFF607710BDC046BC04001010B5054C07
:103B70000021207FFFF7C4FF607F0421FFF7C0FF13
:103B800010BDC046BC04001010B5094C231C8C337A
:103B900018680130FFF780FB064B021CD8620F2328
:103BA0001A4022770211134000126377A07710BDEC
:103BB000BC040010580C001010B5084C0E21201C3D
:103BC00001F09AFA201C0E300E2101F095FA201C0B
:103BD0001C300E2101F090FA10BDC046BC0400104C
:103BE00010B50C4B191C0E311A1C187F1C780133B0
:103BF0002043D8768B42F8D1936E002B08D0064B29
:103C00001B690D2B04D1137F111C29310B705373C9
:103C100010BDC046BC040010580C001010B50C4B71
:103C2000191C0E311A1C1C7F187801332040D876DD
:103C30008B42F8D1936E002B08D0064B1B690D2BDD
:103C400004D1137F111C29310B70537310BDC04672
:103C5000BC040010580C001030B5002185B00E4B8C
:103C6000421C1818007F6C4608550D25D40F181CEF
:103C7000002395425C416442013122400E2901D06B
:103C8000101CECE76C46E15CC218013311770E2B77
:103C9000F8D105B030BDC046BC040010074B10B5CC
:103CA0005A6E16329200D458611E1C19D1502077DA
:103CB000002901DA0D21D15010BDC046BC0400100E
:103CC000034A0023111C943198320B601360704733
:103CD000BC040010034B0122943319684A401A6057
:103CE0007047C046BC040010044A002313678C329E
:103CF0001360034B0122DA607047C046BC04001019
:103D0000580C001010B59E4C0F20A16A9D4A8B10D4
:103D100018408911013852560E2848D801F028F968
:103D2000080F171F234729474731474747353900B1
:103D3000002A3CDB944B9A184032002305E0002A0D
:103D400035DB914B9A184032012393712DE0002A04
:103D50002DDB8D4B9A1840329279DA6625E0081CEB
:103D6000FFF79CFF21E0002A21DB101CFFF7FCFD80
:103D70001BE0002A1BDB844B596E16318900CA50A8
:103D800013E0081CFFF786FD0FE0081CFFF75CFD41
:103D90000BE0002A0BDB101CFFF75EFF05E00C2B8D
:103DA00023DD162B28D1FFF705FE0120EEE0982B2E
:103DB00003D1754B00221A66F7E7982B6CDC382B81
:103DC00003D1714B01205866E0E0382B30DC1C2B0E
:103DD00002D1FFF739FEE8E71C2B12DC0C2BDED1F9
:103DE000694B012098331860D0E00120002B00D1EE
:103DF000CCE001204042C9E0182BFAD1FFF774FF54
:103E0000D3E7282B03D1604B00225A66CDE7282B3D
:103E100004DC262BEDD1FFF7E3FDC6E72C2B02D106
:103E2000FFF71CFEC1E7362BE3D1FFF7EDFDBCE742
:103E3000662B02D1FFF732FEB7E7662B16DC4C2B60
:103E400003D1FFF7A1FE0220A0E04C2B04DC3C2BA9
:103E5000CFD1FFF70DFEA8E7562B02D1FFF714FED6
:103E6000A3E75C2BC5D1FFF71DFC9EE76C2B02D1AD
:103E7000FFF72CFC99E76C2B04DC682BB9D1FFF71A
:103E80009BFE92E7762B02D1FFF712FE8DE7882B7F
:103E9000AFD1FFF785FC88E7E62B02D1FFF758FE8C
:103EA00083E7E62B35DCC82B02D1FFF713FF7CE755
:103EB000C82B16DCA82B03D1334B0120186665E014
:103EC000A82B04DC9C2B94D1FFF77EFC6DE7B82B6C
:103ED00002D1FFF7F5FE68E7BC2B8AD1FFF704FD9E
:103EE00063E7D62B02D1FFF741FE5EE7D62B05DC58
:103EF000CC2B00D07DE7FFF719FD56E7D82B02D178
:103F0000FFF702FC51E7DC2B00D072E7FFF768FEF9
:103F10004BE7F32B02D1FFF71BFC46E7F32B17DC33
:103F2000EC2B02D1FFF77AFE3FE7EC2B05DCE82B08
:103F300000D05EE7FFF7FAFB37E7F12B02D1FFF77E
:103F4000C3FD32E7F22B00D053E7012020621DE0D1
:103F5000F62B02D1FFF7E4FD27E7F62B05DCF52B66
:103F600000D046E7FFF70CFD1FE7F72B02D1FFF764
:103F700013FD1AE7F82B00D03BE7FFF7B7FB14E778
:103F8000580C0010EC990000BC04001010BDC04695
:103F900038B5184C231C8C331868FFF77DF9164B85
:103FA0000022E16EDA60E26603229862A1661040A8
:103FB0001D1C022809D090420AD0012802D0FFF728
:103FC000A1FE07E0FFF726FB04E0FFF7A1F901E0FF
:103FD000FFF74AFB00280BDDEB68002B04D1231C04
:103FE0008C3319680A181A609034226813182360F9
:103FF00038BDC046BC040010580C0010034B012211
:10400000DA660F229A775A771A777047BC04001045
:1040100010B5054C0549201C01F06EF8FFF7EEFFC6
:104020000123636610BDC046BC0400109C0700005D
:104030007047000030B50C4D049C28600B480160AF
:104040000B490A600B4A13600B4B039A1A600B4B27
:104050000B4A1C600B4B1C600B4B1A600B4B0C4A41
:1040600013600C4A136030BD500300105C03001055
:10407000640300103803001030030010100000101B
:10408000D9400000580C00102C03001031400000F3
:104090006003001048030010014B18607047C046D1
:1040A00034030010094B10B51A68191C084B002A7C
:1040B00003D1084C2468226003E01A68904200DAB9
:1040C000101C186001230B6010BDC0463C0300109B
:1040D000580300103403001013B50023009301931C
:1040E000114B124C1A68124B11681868814202D1A8
:1040F0002268009208E012681A600E4B1B68002BC1
:1041000002D0684601A99847009B2360002B04D089
:10411000094A64209361FFF7C5FF009A531E9A4134
:10412000064BDA6613BDC046380300104C0300107E
:104130000C0000105C030010580C0010BC040010B0
:10414000034B1B68002B01D1024A13607047C04625
:10415000440300103C030010014B4A3318787047A9
:10416000BC04001038B5164B1A1C98321268002A8D
:1041700004D0144B1C6801231C4001E094331C68DC
:10418000114DAB689C4202D16A68002A16D0002CFF
:1041900002D1002B0AD111E00C4B1B68002B02D07E
:1041A000201C6968984700236B6006E0074B1B687A
:1041B000002B02D0201C211C9847AC6038BDC046A3
:1041C000BC04001040030010580C001050030010F5
:1041D00008B5084A084B126819688A1A05D5FA22E8
:1041E00052001A60054B1A6801321A60FFF7BAFFD5
:1041F00008BDC0463003001014000010400300103A
:10420000F8B50E1C0E21041C171C00F075FF174B8F
:1042100003259E4211DD092363730123237323E0E9
:10422000301C0A2100F05CFF301C61550A2100F0AF
:1042300001FF0135061C0D2D01D0002EF0D1EF1B22
:10424000033F27706B1E022B05D0E15C621BD21866
:104250005173013BF7E70F235D1B013D6B1C032BE3
:1042600002DD00236355F8E7F8BDC046FFC99A3B5D
:1042700037B5041C0025002300930193124B1B68E3
:10428000002B02D0684601A9984700980135002804
:1042900000D000250220FCF752F80C4B1A680C4B9A
:1042A0001168186881420AD012681A60FFF790FFFF
:1042B000002C04D0013C002C01D1201C02E0032D75
:1042C000D9DD01203EBDC0465C030010380300105C
:1042D000540300100278002A01D180225200437852
:1042E000002B01D180235B00D01A7047F0B59B23CF
:1042F000234D5B00EC5C85B003900E1C002C01D1BB
:10430000802464003023FF33EB5C002B01D1802339
:104310005B0002933823FF33EA5C80235B009C42FE
:1043200003D00F23171C1F4000E007271548FFF795
:10433000D1FF0299421C631A802149000C1B0721FE
:10434000C91B0094019103980F49FEF7B1FB0023AC
:1043500033704124301CFEF7FCFBBA235B00371896
:10436000E818001BFFF7B6FF221C031C0749381C86
:104370000134FEF79DFB462CECD105B0F0BDC046E4
:10438000BC040010F0050010FC990000099A000020
:10439000F0B5564D564C2B1C94331B6893B0061C3D
:1043A000A061E161002B17D118280BD1C32909D1D5
:1043B000504B1B680F2B05D1281C38300E211622BC
:1043C00000F012F9A069182804D1E269332A01D15A
:1043D00000F0B0F8FFF712FE002E02D00A2363614E
:1043E00000E06661444BA069444F18603B68444E4E
:1043F0001B683360FFF7A4FE012300222B670192A4
:10440000404B1B68002B1AD03F4E3368371C002BE3
:1044100015D01B68002B04D13C4B1B6898473B68A8
:10442000F7E733681A68013A1A60394A1368002BB3
:1044300005DD013B1360002B01D1FFF781FEFFF783
:10444000A7FD002801DAFCF72DF8324B01989842BD
:1044500005D04023021C9A432F4B9A420BD1A36AEA
:104460002E4A934204D0082293432D4A934202D10C
:104470000A20FFF717FEA26A2E1C8C3601923368C1
:10448000284A934203D0284A93420BD019E0FFF701
:1044900069FEFBF783FF1A4B19481B680093013B29
:1044A00003600EE0214F3A68002A0AD002A80AA948
:1044B000FFF71CFF3B6802A80AA998473368273317
:1044C00033600E4B1A681A4B11681868814206D087
:1044D00012681A60FFF77CFE0C4B1B6898472A6F26
:1044E000002A8DD1FFF73EFE13B0F0BDBC040010D2
:1044F000580C0010100000104C030010380300107E
:104500000C0000103C030010340300106003001086
:10451000580300106E02000026020000FB0300009A
:10452000E3030000790D00003E2700006403001043
:1045300054030010F7B5274E002033681C68FFF7BE
:1045400097FE33681A689442FCD01B6801272D330C
:10455000FF330193FFF752FD1F4C0A231F4D636188
:104560001823A3611523E3612B1C9033002267629B
:104570001A60FFF743FD2F673368019A1B689A4260
:104580000CD0FFF705FD3268154B116818688142A1
:10459000F2D012681A60FFF71BFEEDE72B1C012713
:1045A0009033182000211E686762FFF7F1FE0D4B63
:1045B000301C196800F03EFD3835011C0422281C0F
:1045C000FFF71EFE1823A3610023301C6762E3611E
:1045D000FEBDC04638030010580C0010BC0400108B
:1045E000540300103003001070B5002A10DD047869
:1045F00001231C404B1E002B08DBC55CE4006E0849
:104600003443C4540124013B2C40F4E7013AECE765
:1046100070BD30B59A4205DC845C8D5C85548C5449
:104620000132F7E730BDF0B5069E051C07A80478F7
:104630003078002A17D0059EB34217DCCE5CD75CD9
:10464000F7193F180020A74201DB3F1B0120EF5460
:104650000133F0E7CA5C12180020A24201DB121BF2
:104660000120EA540133059A9342F3DD01231840F7
:10467000069B1870F0BDF7B50AAC2478099D00942C
:10468000089E2C7800282DD0002928D0002A18D088
:10469000B34248DCCF5CD55C7F1B3F1B0024A742A4
:1046A00002DA009C3F190124C7540133F0E7CA5CC9
:1046B000121B0024551C02D1009A0124013AC25455
:1046C0000133B342F3DD2EE0D15C4942091B0024E3
:1046D000A14202D0009F0124C919C1540133B34241
:1046E000F2DD20E0002914D0002A08D0B3421ADC01
:1046F000CD5CD05C0133281A041BE40FF6E7B3420B
:1047000011DCCA5C0133141B013462425441E4B22F
:10471000F5E7B34207DCD15C013349420C1B611E53
:104720008C41E4B2F5E701231C40099B1C70F7BDE6
:1047300070B5049C0125257000290BD09A420BDC32
:10474000865C8D5CAE4209D10132F7E7815C0029BD
:1047500004D101329A42F9DD0023237070BD9142E9
:1047600004DA43185B7843540131F8E700234354DB
:1047700070478A4205DD8318013B1B788354013A58
:10478000F7E7002383547047F7B5134A134C1378A7
:104790005278C35C134000D040231149236012318A
:1047A000009100220023A6187360009B0125123B94
:1047B0001F785978C75D394202D077682F437760F8
:1047C000009F02336D00BB42F2D1123304320093DA
:1047D000282AE7D10020FEBD04010010180E0010A9
:1047E00050000010122330B54B43334A0131D31827
:1047F000052251431A785C78825C144204D02F4A17
:104800005F245218947054709A78DC78825C144259
:1048100004D02A4A7C245218533214701A795C79D5
:10482000825C144204D0254A7C245218A3321470AE
:104830009A79DC79825C144207D0204C5F2264189C
:10484000251CA235A1342A7022701A7A5C7A825C07
:10485000144204D0194A7C245218A03214709A7A57
:10486000DC7A825C144204D0144A7C245218503200
:1048700014701A7B5C7B825C144207D00F4C5F2261
:104880006418251C523551342A7022709A7BDC7BC7
:10489000825C144204D0094A2E245218A4321470A7
:1048A0001A7C5B7C825C134204D0044B5918F431AF
:1048B00027230B70002030BD50000010880C001022
:1048C000F8B52E4D061C00272C1C281C20214F2239
:1048D000FEF71CF9002F04D02A1C7C2339322B70E0
:1048E00013702B1C4F33002201371A705035052FDF
:1048F000EBD1211C2D2338310B70211C37310B706B
:10490000A121A370637049005F2363544221FF31EA
:104910006354A32149006254194A11785278715C9A
:104920000A4204D0221C53325234137023700024E4
:10493000211C301C0134FFF755FF0A2CF8D100244C
:10494000104B114DE25C1B19B15C58780F4A6300A3
:10495000084201D0D15805E0D058FEF7FAF80C49CA
:10496000091A0A31281C023400F0D0FB122CE7D1BE
:10497000281C084900F0CAFB0520F8BD880C00106F
:104980000401001018000010C80D00102C000010C9
:1049900006010010119A0000F0B587B00390FCF7F3
:1049A00097FC8F498F4C029100270C257D43002FE7
:1049B00000D101258C480368032B02D0042B10D0B2
:1049C00002E0874A02920EE0022B0CDC0668012E00
:1049D00000D10DE1022E00D18FE1002E00D0ECE1DC
:1049E000A8E0824B0293002305AA537023687F211D
:1049F0000B405C2B00D194E027DC382B00D18AE0FF
:104A000011DC072B68D005DC022B00D190E0062BCF
:104A100040D0DBE7212B00D181E0232B00D184E0C3
:104A20001C2BD3D17FE04F2B50D007DC3F2B64D021
:104A3000402B64D0392BC9D1432377E0542B74D059
:104A40005B2B41D0502BC1D169E0732B65D00FDCBB
:104A5000662B3DD004DC5E2B55D0622B63D0B5E7CE
:104A60006F2B3DD0712B52D06D2BAFD135235DE034
:104A7000792B4AD006DC762B4BD0772B41D0742B88
:104A8000A4D146E07D2B25D07F2B27D07C2B9DD138
:104A900042234BE031231370022F00DCB8E1231CCA
:104AA000083B1B68194054290AD0032F00D1AFE1FD
:104AB000231C0C3B1A687F231340542B00D0A7E122
:104AC0004C2205AB1A70A3E132232FE033232DE0F3
:104AD00034232BE0362329E0372327E0382325E051
:104AE00039231370062F00DC92E1231F1B68194045
:104AF0004723232900D08BE118E0302316E02D2333
:104B000014E0412312E0442310E045230EE0462345
:104B10000CE048230AE04C2308E0502306E052232F
:104B200004E04F2302E0552300E04E2313706FE1B1
:104B30004923FBE721680123194205D0A81CC0B214
:104B4000311C0522FCF73CFC2268920706D5E81DC3
:104B50000121C0B20A1C0323FCF732FC21680423A4
:104B6000194205D0E81DC0B205210122FCF728FC3E
:104B70002268120706D5A81CC0B20921052201230C
:104B8000FCF71EFC2368DB0606D5681CC0B20521B5
:104B900001220423FCF714FC2168890606D5681C51
:104BA0000121C0B20A1C0323FCF70AFC226852064A
:104BB00006D5A81CC0B2042105220123FCF700FC85
:104BC00023681B0607D5281C0930C0B20921022220
:104BD0000123FCF7F5FB2168C90500D4EDE0E0E016
:104BE0008C5A0000180E001014010010945A000096
:104BF0002268324211D0EBB2181C02300193C0B2CD
:104C000000210522331CFCF7DBFB0198311C03302B
:104C1000C0B20322331CFCF7D3FB216802221142ED
:104C200005D0A81DC0B201210323FCF7C9FB2268EF
:104C300004231A4205D0A81DC0B205210222FCF7A8
:104C4000BFFB23680826334211D0E9B2081C0230AA
:104C50000191C0B2092105220123FCF7B1FB0198A3
:104C6000311C0330C0B203220123FCF7A9FB2268E8
:104C7000D20606D5681CC0B2052102220423FCF727
:104C80009FFB23689B0606D5681CC0B20121022247
:104C90000323FCF795FB216849060ED5EEB2B01C44
:104CA000C0B20421052201230336FCF789FBF0B2D0
:104CB000052103220123FCF783FB2268120607D596
:104CC000281C09300222C0B20821131CFCF778FB13
:104CD0002368DB0571D5EDB22E1C0A36F6B2301C06
:104CE000082102220323FCF76BFB0935301C0B2142
:104CF000FCF752FBE8B20B215DE02168C90706D53D
:104D0000681CC0B200210722331CFCF759FB236842
:104D10000222134205D0A81DC0B200210623FCF7D1
:104D20004FFB226804210A4205D0A81DC0B202220E
:104D30000623FCF745FB236808210B4205D0681CBD
:104D4000C0B207220223FCF73BFB2168C90606D547
:104D5000681CC0B2042102220623FCF731FB226842
:104D6000920606D5681CC0B2002102220623FCF779
:104D700027FB23685B0606D5681CC0B20421072206
:104D80000223FCF71DFB2168090607D5281C093002
:104D90000222C0B20821131CFCF712FB2268D205C4
:104DA0000BD5EDB2281C0930C0B20B210A35FCF737
:104DB000F3FAE8B20A21FCF7EFFA013704340B2FBB
:104DC00000D0F2E51F4B1B68002B05D01E480021C8
:104DD00009221E4BFCF76AFB1D4D00240235AB1E59
:104DE0001A7803996B1E8A5C1B78134208D0194B02
:104DF000A200D058184B0922E15C144BFCF756FB7B
:104E000001340235092CEAD1FCF76CFA07B0F0BD89
:104E1000002205A8291C029BFCF748FB2268120609
:104E200005D5E91D0D480022029BFCF73FFB2368D6
:104E3000DB05C2D5E91D0A480022029BFCF736FBC0
:104E4000BBE7C046440100101B9A0000845A0000D2
:104E50001800001018010010749A0000755B000023
:104E6000199A000038B5FFF777F90624002805D114
:104E7000FCF738FA38BD01340E2CF9DC0321201C74
:104E800000F0D8F80321C5B2201C00F029F9281C35
:104E9000C9B2FCF781FA092CEDD10B24EEE7000032
:104EA00038B5041CFFF770FC201CFFF775FD094B9B
:104EB0001B78002B0DD0201CFFF702FD064CC823E9
:104EC0005B00E518211C05485034FDF7E5FDAC42B8
:104ED000F8D138BD70030010880C00109B52000000
:104EE00000B589B000280ED0FCF7BDF901A8092152
:104EF000FEF7E4F9684612300A21FEF7DFF901A84F
:104F0000FFF7CEFF08E0FCF7B6F9044B1B78002B47
:104F100002D00348FDF7C0FD09B000BD70030010CA
:104F20001D9A0000FEE7FEE708B500230B4A0C4976
:104F30009A188A4204D20B49C95C01331170F5E713
:104F4000094B0A4A591C013B934203D200221A70B2
:104F50000B1CF6E7FBF748FEFEE7C046000000101A
:104F60003C0100107D9A00003D010010440E00102D
:104F700002B4714649084900095C49008E4402BCEC
:104F80007047C04603B47146490840004900095AB9
:104F900049008E4403BC7047002934D0012300220D
:104FA00010B488422CD301242407A14204D28142A8
:104FB00002D209011B01F8E7E400A14204D28142B8
:104FC00002D249005B00F8E7884201D3401A1A4335
:104FD0004C08A04202D3001B5C0822438C08A0426C
:104FE00002D3001B9C082243CC08A04202D3001B22
:104FF000DC082243002803D01B0901D00909E3E79C
:10500000101C10BC7047002801D00020C04307B41A
:10501000024802A14018029003BDC046D90000001A
:105020000029F0D003B5FFF7B9FF0EBC4243891A3F
:105030001847C046002941D010B4041C4C40A44677
:1050400001230022002900D54942002800D5404212
:1050500088422CD301242407A14204D2814202D2E7
:1050600009011B01F8E7E400A14204D2814202D207
:1050700049005B00F8E7884201D3401A1A434C0804
:10508000A04202D3001B5C0822438C08A04202D33A
:10509000001B9C082243CC08A04202D3001BDC0862
:1050A0002243002803D01B0901D00909E3E7101CA3
:1050B0006446002C00D5404210BC7047002806D042
:1050C00003DB0020C043400801E08020000607B455
:1050D000024802A14018029003BDC046190000001A
:1050E0000029EBD003B5FFF7A7FF0EBC4243891A96
:1050F0001847C0467047C04642180023002903D015
:10510000037001309042FBD17047C04670B5061C59
:10511000B30717D133680F480F4D1A189A43301C44
:105120002A420FD1043002680A4BD41894432C420F
:1051300008D104300268074BD41894432C42F1D0B4
:1051400000E001300278002AFBD1FDF70BFD301C96
:1051500070BDC046FFFEFEFE808080802573202546
:10516000730D0A00444D31355F4D383000534552C0
:1051700049414C20434F4E534F4C4500726561648A
:1051800079000D0A4279652E2E2E0D0A004E4F0031
:10519000203F002573202573202025694D485A00A3
:1051A00056323600202025692E25303369560020DE
:1051B00025735254432000444D343100444D343162
:1051C000204F4B0020204552523A20256900424191
:1051D00044204B4559202530327800202D202530A1
:1051E0003278004C43443A25303269202D2025691D
:1051F00000505245535320454E54455220544F20A1
:10520000534156450053495A453A2569205553455F
:10521000443A256920465245453A25690053544190
:10522000434B3A0025633120484F5552002D005220
:1052300054432052454144204641494C0074757204
:105240006E6564206F6E003C52455345543E0D0A16
:1052500000426164206E756D6265722E0D0A004217
:1052600041543A2025696D560D0A000D0A25303249
:105270007820200057616974696E6720666F72201C
:10528000646174612E2E2E0D0A00426164206D6FE0
:1052900064656C0D0A00526561642025730D0A0077
:1052A0004641494C4544006F6666004C43442064C7
:1052B000656275672025730D0A00436F6E736F6C0E
:1052C000652074696D656F75742073657420746FE3
:1052D000202569206D696E757465730D0A000000E4
:1052E00000005C000C000C7C287C7C447C24104872
:1052F000285408000C0038440044380020100810DE
:105300003810804000101010004000201008384471
:1053100038007C006454484454281C107C4C5424AD
:1053200038542004740C2854280854380050008045
:105330005000102844282828442810045408384CC9
:105340005C7814787C54283844447C44387C544439
:105350007C14043844347C107C007C0020403C7C6D
:10536000106C7C40407C087C7C047C7C447C7C14FD
:10537000083844787C1468485424047C047C407CBD
:105380003C403C7C207C6C106C1C601C64544C7C4D
:105390004400081020447C00080408808080040831
:1053A000007844780007080400000000BF01BF0136
:1053B0000905000007000700070007130A00002086
:1053C00000E400FC003F00E700FC003F0027000471
:1053D0000F0800000C011E01FF03FF032201E20180
:1053E000C2190D00000E001F0011019101FF007E87
:1053F00000FC00FE0113011101F001E0140A00009D
:10540000EE00FF0111011101BF01EE00E0013001CA
:105410001001050300000F000F0A050000F800FE50
:1054200003070701040B060000000001040707FE44
:1054300003F80F08000000000A000E001F001F0004
:105440000E000A11090000100010001000FE00FEFE
:105450000010001000100804000000048007800302
:105460000D070000100010001000100010001008C0
:105470000400000000800180010D07000C000FC037
:1054800003F0003C000F00030F080000FE00FF01C6
:10549000010101010101FF01FE10080000000002EE
:1054A000010201FF01FF0100010001100800008658
:1054B00001C7016101210131011F010E010F080027
:1054C0000082008301110111011101FF01EE110998
:1054D0000000300038002C002600FF01FF012000F2
:1054E000200F08000080009F011F0111011101F130
:1054F00001E10F080000FC00FE010B010901090198
:10550000F901F00F08000001000100C101F1013DA7
:10551000000F00030F080000EE00FF011101110150
:105520001101FF01EE0F0800001E003F01210121C3
:1055300001A101FF007E0804000000008C018C0125
:105540000804000000048C078C03120900002000EE
:1055500070005000D80088008C010401040111097A
:105560000000480048004800480048004800480043
:105570004811090000040104018C018800D8005082
:10558000007000200D07000002000300B101B90106
:105590000F0006190D0000F800FC010603FB06FDD4
:1055A0000505050505FD05FF050601FC01F81209C5
:1055B00000008001F0017C004F004F007C00F001F2
:1055C00080010F080000FF01FF01110111011F01FF
:1055D000FE01E0110900007C00FE008301010101D1
:1055E00001010183018211090000FF01FF01010196
:1055F000010101018301FE007C10080000FF01FF92
:1056000001110111011101110111010F080000FF29
:1056100001FF011100110011001100011209000029
:105620007C00FE008301010121012101E301E2016F
:1056300012090000FF01FF0110001000100010000F
:10564000FF01FF010A0500000101FF01FF01010147
:105650000B060001000101010101FF01FF1008001C
:1056600000FF01FF0138006C00C60083010101103A
:10567000080000FF01FF010001000100010001001E
:1056800001160B0000FF01FF010F003C00F000F0CD
:10569000003C000F00FF01FF0112090000FF01FFA5
:1056A000010F001C007000E001FF01FF01130A0060
:1056B000007C00FE0083010101010101018301FE64
:1056C000007C0F080000FF01FF01210021002100E4
:1056D0003F001E140A00007C00FE0083010101014E
:1056E0000101038307FE047C0412090000FF01FF8F
:1056F00001210021007100DF008E0100011109006D
:10570000008E009F011101110111011101F301E24D
:1057100011090000010001000100FF01FF0101006B
:10572000010001110900007F00FF0080010001005D
:10573000018001FF007F1109000007001F007800B1
:10574000E001E00178001F0007190D00000F007F45
:1057500000F001E0017C001F001F007C00E001F070
:10576000017F000F120900008301C7016C0038009F
:1057700038006C00C7018301110900000100070017
:105780001E00F801F8011E00070001120900008147
:1057900001C1016101310119010D0107010301007E
:1057A00004040200007F010905000007000000005A
:1057B00000070B064400FF0144004400FF01440BB6
:1057C0000600008C001201FF032201C40D078200B5
:1057D00045002500920048014401820C060000E6C5
:1057E0000019012601C0002001070400000000018B
:1057F0000002080400000000FE010102080400008D
:1058000000000102FE010B0600008800500020008D
:105810005000880B06000020002000F80020002027
:1058200006030000000400020B0600002000200018
:1058300020002000200603000000000001090500F0
:1058400000800160001800060B060000FE00010148
:1058500001010101FE0804000002000200FF010C2A
:1058600006000082014101210111010E010B060019
:10587000008200010111011101EE0B060000600021
:1058800058004600FF01400B0600009F0009010977
:10589000010901F10B060000FE00110111011101C7
:1058A000E20B0600000100C10131000D00030B06F0
:1058B0000000EE00110111011101EE0B0600008E37
:1058C00000110111011101FE0804000000008C010B
:1058D0008C01080400000000000208010A05000015
:1058E00020005000880004010B060000500050000A
:1058F00050005000500905000004018800500020AD
:105900000B06000002000100610111000E0D077876
:1059100000860132014902390242027C0E078001F1
:1059200070004C0043004C00700080010B0600002A
:10593000FF01110111011101EE0B06FE0001010131
:105940000101010101820B06FF01010101010101B9
:1059500082007C0C060000FF011101110111010100
:10596000010B060000FF01110011001100010C06DF
:10597000FE000101010111019100F2010C06FF017D
:105980001000100010001000FF01080400000000CB
:105990000000FF010704C00000010001FF0E070026
:1059A00000FF01180024004200810000010C0600E5
:1059B00000FF0100010001000100010E07FF010CC2
:1059C000003000C00030000C00FF010C06FF010693
:1059D0000018002000C000FF010B06FE00010101BD
:1059E0000101010101FE0B06FF0111001100110070
:1059F00011000E0C06FE000101010141018101FEB2
:105A0000020C06FF011100110011002900C6010B54
:105A10000600008E00110111011101E20B060000C9
:105A200001000100FF010100010B06FF0000010061
:105A30000100010001FF0D0703001C006000800150
:105A400060001C00030D071F00600080017C0080C7
:105A50000160001F0E078301440028001000280089
:105A6000440083010D07030004000800F001080052
:105A70000400030E07810141012101110109010503
:105A80000103010003072061DE5200000D0C205AC3
:105A90009F5700000D0C205AA45300000007000877
:105AA000000A010018111013383130337871707307
:105AB000C8C1C0C38881808384848782C5C4C7C2AB
:105AC00075747772353437321514171202070208CD
:105AD0000201000301090304020402050305000694
:105AE0002024282C383C4044484C4669726D77612C
:105AF00072652025735F5632360D0A00252D313030
:105B0000732025732573000D0A5479706520273C96
:105B1000636F6D6D616E643E203F2720666F72205B
:105B2000706172616D730D0A00557074696D652046
:105B30002575730D0A0025730D0A0D0A00564F597D
:105B400041474552203E3E200025630048656C7069
:105B5000004E6F20706172616D73004B657920702B
:105B600072657373003C6B6579313E203C6B6579DF
:105B7000323E202E2E2E0044756D70206D656D6FA7
:105B80007279004C6F6164206D656D6F727900638E
:105B90007400436F6E736F6C652074696D656F750B
:105BA00074003C6D696E757465733E0047657420C2
:105BB00074696D65007473005365742074696D6554
:105BC000003C595959594D4D44443E203C48484D9C
:105BD0004D53533E007464005570646174652074C5
:105BE000696D65003C6F66667365745F696E5F6DB5
:105BF000696E757465733E00546F67676C652064E9
:105C00006973706C6179206F757470757420746F2E
:105C100020636F6E736F6C65006200526561642073
:105C20006261747465727920766F6C746167650067
:105C30009151000000000000DD1B00004C5B0000E3
:105C4000515B00004F5B0000FF000000AD10000042
:105C50005B5B0000655B0000AD5D000000000000C4
:105C6000D10E0000775B0000515B00003B5D00003F
:105C700000000000710F0000835B0000515B00001A
:105C80008F5B00000100000031110000925B0000FA
:105C9000A25B0000905B000000000000F90D000016
:105CA000AC5B0000515B0000B55B0000020000002F
:105CB000590E0000B85B0000C15B0000D55B00001E
:105CC00001000000990E0000D85B0000E45B0000BA
:105CD000D65B00000000000005110000F85B00002A
:105CE000515B0000195C000000000000E50D0000A1
:105CF0001B5C0000515B00000080015000800250DE
:105D000000800350FC3F0150FC3F0250FC3F035019
:105D10002578000D0A413A2000202025633A200012
:105D20000D0A533A20000D0A4D3A20002020473A30
:105D300020253032780D0A006661696C0025303408
:105D4000692D253032692D253032692025303269A0
:105D50003A253032693A25303269202573002530E2
:105D600032783A253032783A253032692E25303271
:105D7000690025303278203A202569202569203AAB
:105D80002025303278004E4F2052544300253032C7
:105D9000783A253032783A25303278002530347818
:105DA0002D253032782D25303278202025730000C3
:105DB000D05D0000D45D0000D85D0000DC5D000017
:105DC000E05D0000E45D0000E85D00003C5B000079
:105DD0004D4F4E005455450057454400544855001A
:105DE000465249005341540053554E00CCC5ED2D49
:105DF0001207EE76A609CFA6C6FC205FFD8D14160D
:105E0000A5B8757A3E3979BAAC30388E4526243C2F
:105E100071EA4D1DFC6918F8374D202D5431210CC5
:105E20007B81EFB98C658A36C3DF9BAF1E308AD683
:105E3000E807680B0BE035688B58BB367E32A97AD1
:105E40000BFA57FD0296BF98D0985FEC4861E9BA0B
:105E5000233F67B933A85C1D8A2E7C20E734A69EB9
:105E6000180B638521022479A02300408133DC9440
:105E70002FFB993C5492B0BE5BC9D31C43B1DDD813
:105E800082327602251407C50DB09AA840A8A51E37
:105E90003236A06AEE5A06EA4519274A15D2450459
:105EA000CCA2AA4A45069C91AC0C91595B1630E1F4
:105EB00089E8685DA5CC18E5F9AC69CE6D5B5875CD
:105EC00037C847ABC306D05F490DF7D3728C03EEDA
:105ED0006C76DFD400858D59558EDC03D6F46B0DBE
:105EE000ECD3879CB706E117A13110ECD4887F1F53
:105EF00010CA9FC23E76045EA638315A0F194981F6
:105F00002919BDDE16F74461A154A2E5ED29ADA61D
:105F10006BBA4C0BB86D36E573F542257B305B05EB
:105F2000AE43AA9562856B34907EA481B93B4366EB
:105F300044837252D0B598FB7C73D92076A23A8202
:105F40007F51C2274FDC7FBB8A9ACD3FBD4DDBE737
:105F500078C921983DCD24CD2698FB0B4161E9A657
:105F60005592AE9DC6A681AAC9E86FCA34249BA2E9
:105F700039A3319056AC2FFE5593AB5EAFDBAC7AB4
:105F800001AF54C3A8139848C08E2DB66DAB4451D1
:105F9000B708D9D9B9AF415329EDC908A857FF4C63
:105FA000E03F2A595B084DCBD85EE3F04527E20479
:105FB000E16D1CBEF4C273E99F818CF866229A6D74
:105FC0000C32D98B088E4F8419611A2FC61CFC2203
:105FD0005919B13550CADEB8B48E39C586527769C1
:105FE00010C4E319A4391728409DE89C34CDE74E2E
:105FF000FDA3AB571ACDE49B6787A4D6975534F918
:10600000F710871B6628B1090B342D9697B2EE0A5C
:1060100076879DEFC602940373943DD9D2F69ABD5C
:1060200050E96EA6D70ABAFCBC8E6E45B0AFC5DD8E
:10603000D821FF448AEF678FD6D734C920A68C6D4C
:10604000C459CD6C6D5171B1691A45A79C15BB56E9
:10605000A10CF2318E1A0411C7EED93DCA1EEF4DC4
:10606000E5F968A3B5D55CC5C16A188675FAF9D596
:1060700004F07A5F87DB52FBF97AA23B5516D08990
:106080008DC96CDC7C1E596FF86C154829CA4820F4
:10609000B8C0DC4D72A4F7ACA54A4DED02DE7E4ED1
:1060A0009E8727BDC8F7A2658A4FE9ECE338336FB6
:1060B0006BB7B8AC9AA5FD068DE255B7BD0D51CAB8
:1060C000DBF620490882928C113F4632852BBC13A7
:1060D000E8B2B557CDD73C090B6F55A3BA423D2B5B
:1060E000E47A8C769718A79840096154979F931388
:1060F000418D0E5A1D57932772739799AEC133EF96
:106100004604FB402A8991186AF0D8C200D6DAD931
:1061100084DCCEACB8379BFFA463D0F25F862682C6
:10612000331593FA87F931DD495CB55DAA46C9A7F5
:10613000D3C5A3CAC2735E9E8018CD4C2D6B9ED66C
:10614000C325B1365C49024F0FF606057FC5E755FA
:10615000C164E8195A8C5C4C404610087EC4DF9C30
:1061600072CB42BB1362993AE4DDEA19E28C6A59B8
:106170005AF60D3430784D88A93DF8F0BD47D88FD8
:10618000CF48814A793F42D30B3E4CD3376D49F11A
:10619000DCD59909198CF57D6F5688B98AAC2246F1
:1061A000751DB5B6DD07FC115E295A04A40861B45B
:1061B00092D62117D06BD871719BE3A4D0A5C4E50A
:1061C000F091CEC357A5A372F926EABE6A72FF8288
:1061D000447D6E09FC643D54AC8B607D51072167A2
:1061E00081A1FDEFEDF97896CA84E72BA8BD65691A
:1061F00000AEA6C08BF25EF5D21A1C5E6B2D87E155
:10620000EB4331A0E997540A55920BC633B8DEE44C
:10621000C2451C86EF3B9B8D38A25BF5A2EDDE5597
:10622000A4EC8A18EBD67D26EB364049A1FAACC522
:106230000DC5FC8B9D077F22F38D36ADE521A2A411
:10624000BA10E1ABDE01B9188C23F48940BB13719D
:10625000814A394D36E8BE4F2E509D0097C1B57921
:106260004BB852B4A196006A8E8BE47803D5E2DC79
:1062700039170B3E9084B824B2A9F11D3957D43791
:1062800015BD754290AD8BD8BE099505E7FAE5B10D
:10629000C667D7B191BC1ED46A671C2421EBAE6AD5
:1062A000D89143F3E317B6E4B0630AF6BE016F1664
:1062B000FF8EB9BFB3723A54A98E35FD033FBB9E22
:1062C000CA6FA48BC3F343F5A07EA4DCFD2761C194
:1062D0001C0CE16A7F2CA21A3583B9517A9F471DA5
:1062E00014855E84E39F79513CE363398D718F613E
:1062F000DAEA2251E7A255A199F1EA8986939C2B0B
:1063000052DC0E89DCE2862C8749E4B88F223F906C
:106310007DE7EF369B12BE3D57610D255CD43CEE08
:106320009E28859E6278FDD97E4C5942F93367A537
:1063300086177D307E019A0DE2E21A30C2F0016FBD
:106340003E9AF120D926F10CC37C59DBCAC16B9768
:1063500006164EC7C61E1E958EEC8987092D343A47
:106360000056B5C6558F2B6456D5933D7586185586
:1063700030533627CCC5E4CD05822759FF5FC05383
:106380001407A7DF57CC3208DD665203718EE00494
:106390008E78A02F2BDCD8302427DE6822FA8617CF
:1063A0002E26902434CD9ABAF7BE64D7E68B3749AF
:1063B000A3E2905C798382609D4A1F0CC0994602DB
:1063C00063AE72E10F9472FB1BC17363F6E2D930C6
:1063D00096439D0E3D180A672762FCC95BB0C263F5
:1063E00008C0AA8F51E44A4DEC6FF3CA22371E91C0
:1063F000ADA047E8BDE8EB903DB1B0452B4F021C86
:106400004FFD5C18A8B35EA7BE55D5B98568EA589C
:10641000E8F308BF02B2FA579E96342A2C30C63EE3
:10642000DD136A92D83CA61EB90CD096B1ADBD1052
:10643000B890673EF4B68D4D200E15607FDC813834
:10644000D2E58A85AFC1A8EF2D0BAC92344346E963
:10645000718546AF20B3EB0E3AC8332392D1C0F515
:106460001F4EEE0C54B6FBDBD4FFF4C3755A06295D
:106470001518B8EEE93A52F2DB370C7BB332FFE085
:10648000EC03A857E58FB6CBBD9377500DEA3EE7F6
:10649000FDF697AF4E1394C31B5426E1914FCEEBFC
:1064A00043E9997C8E4AC28DD6C2EBCFF311765A5E
:1064B000A26BF083EBAAC386858A744DAC32B176A9
:1064C0006C981BEE7C1B5E7A31A29D8164A0FF213B
:1064D0001A43C92E56E2155BD51DF426143E0CB1A5
:1064E0008AE207A477861D0D061177E95B10FC2F61
:1064F000E4B58C0B6C676FEB26C2F7662E4F8D826E
:1065000039D4F16C66470A642605590AB983B8DBA9
:10651000A73FF50987063C67064219135293F7A572
:10652000B694D07C96186B4674BA8BAD36AB2A986D
:10653000A2FB6F42B1F42D034AECB88727BF95B98F
:106540002BE53197A16990C25145CB2F0FF4313B18
:10655000EB232E0C58CC507E1A13FAC6524ED1D4CF
:106560006A417B048FF176BE8F0068128C5FAECEDD
:10657000046B19D1DE1068718B65A472F36D5784BA
:10658000586169DF2787A014E6EDEFCD94AF72A7BD
:10659000FB6CD6E86220B90676DFA9DE3071AFBAAF
:1065A000000E82560F9C9476484DAB9CB87B47A555
:1065B000A7758FCC73C5D4E393E02DBB872A37D45E
:1065C000A282768FFF915B5ACEBCF4BEA5B6107B3B
:1065D00052FB43B02E8F1EF5F8215A573C0A7F2BF1
:1065E000AF5227BD64283C5C0522E9D5F09B476685
:1065F00060D06DA6AE85BA17ACE316FEF331BF8747
:106600006524F7C51EB459476DC326C6F0FE240D98
:10661000EFDA60108B9FB70B989A9DA84FE131F489
:106620005E1BBA37B4E15A8D94A77E6167AD49D03D
:106630007124513B16F9057530762087EEFAF4DCAB
:1066400065C7315F19064602CDA58779DADCFE3CC5
:106650005AB14080EA4132C816CC97992545BFB25D
:106660002F70B3A4683E5BB591B13DADE7182B34F4
:10667000B446AE5CB6ABC5997195BA5C57621980E9
:1066800081E27CCEBD8C12622B2AC00A40A61AEE93
:1066900079F06BF69B2F393EA7E643894B6233B402
:1066A000DFB0DD983DB0A0F60C502238708E9FA769
:1066B000251AEE4543E7C36F56BF1548704B6D9ED4
:1066C0009599C82269D6283878095EB7F6AB9C80C0
:1066D000DDC82E32783A9CFB26E02DB57B5F9C1DF1
:1066E000589BDF9AFA1ED8E677C5802A55CB7F7370
:1066F00055AF3138A0CCD322E7C416215089761388
:106700003010BCFA861B2990FBF0EB4784A67DE095
:1067100096BDF77137C91B9F45F1312410B10508AB
:106720003474342535D17CAE6695698A315CEC1DB4
:1067300082F729E57F93CB24B687B96980A6987F35
:10674000B8676C8E7CDC9B395C921988ABB8EE36EE
:1067500021B19240CAFC813958F0F9654EDBBCCEBC
:10676000D225B7B47DC0315051B1C8B5BFE321C007
:106770002E8304176068A78D363618152BC28BB789
:106780009E3BD19FBB8B7506281C6635C6A37D66D4
:10679000B00E3A228B7D57446CDA241A0E569D14A3
:1067A0008F6B18D303FD168601A00055D043329A93
:1067B0004E0933A506265689D49DE5C82F1306C079
:1067C00032A839BDD65988400FFD57C2DFBA9BBBEE
:1067D0003163F885C4CA5B2E719BBE3D5256E00AF8
:1067E000D00EE94D748E454345913410EC34861932
:1067F000B58563FFB8755CD67577ADDCA60C07214F
:106800000767DE6EBEC49368B3275606351822CBE1
:10681000E4686E4A597BECD0A2A7023521C72FA3AA
:1068200009D47B26D5A9898DE5FD5AA948CAD40D7E
:1068300023A016A9F90AB56B49F6589FCFDA88C488
:106840004616C0DFF24B159B84BB90198322CA49C0
:106850007D6C5030E3A9CCEE2BE772086F2994864B
:106860000C1106351281A54813CE270C9281370BE7
:10687000884F4489702E69A8D116703B2D76A8F9EF
:10688000D44FBB9E841558F89D363B6E68C9627D17
:10689000C38A75120419A65A77A3476A6C660CF16D
:1068A00075113F197A6A260F56454E36597C3E437C
:1068B00056F1CDF751635D7A671FD97BF895A4FD3A
:1068C000908E54990E1FD2683982359F13201E93E3
:1068D000D05DAB11D69AFDAC0B69F4AC1E5D7E0D9C
:1068E00082E59D77BED085CC936EDFD7BE8B367C9C
:1068F0009F04739EE9875B58A8D8822861D9C10597
:10690000761212E662F735F5FA1911D53165DB48D2
:10691000F9C4A5C8FE76EFE17461220A35ABC5E67D
:10692000B13DE74EBB1BC0D330247C3E5049ECA5A3
:106930001D4387BB97DEB34FD8415ADDD366D5716F
:10694000BB9D062D750BB76C3C0FE76003BF3BBECC
:10695000BD3C1782EE4C524AD9FB66FE48862CC9D4
:10696000F8BFF84440F867D795517B7A970596C1F0
:10697000F7E9C1F5B9F3D6F78A9EBB97E8B03619A7
:10698000EAD6FDCEF7A8B6960A1E97A9FF5B78D582
:10699000054F9F665C9460331A2C8EBEAD473E79DE
:1069A000B0B7071EFFBB11C5FE4D74491C02AC1EDB
:1069B0001364BA0AE18F003010E32F57038D7E9BDA
:1069C00079A3055C1AE8B600C5EF06E0A073E444BD
:1069D000BBB5EE5E1C58954B033EDD42987567963D
:1069E000EB2B13C8303B5916CDC9F260E82A8E0D47
:1069F000CC84798804EE306EC923B8C493D8B4B17E
:106A0000AF09611C20CB7FB5B8685E3DC0EC772034
:106A100042C4D6C5BC8B5F7114405B6AB9B3D75B07
:106A20006BC0D021CDD8A55F446EB28E8AEC76F3D0
:106A30008B0EDE8B68A8EB608B0B65E7711EE0B6F2
:106A40002BCCC274685ED81F628CC85FFD776FD88C
:106A500055DC56FD1F6FBB153AF11DA3F0575318B7
:106A6000C681E10AB9929EF5B8D9C7FEE37A255BE3
:106A7000B14E259723D1C4C07A542EE926050C586F
:106A80008641D7157632A4BFFC7FB60A65A02EA139
:106A9000EB27FB010AEB7D00E2A01F355A0DAF6B1F
:106AA000C9CC2332BF95099E77E799A515FE5604F8
:106AB0001D81FFEDE66E3171944AEEBCC0E6DEDC6E
:106AC0005405C33A4EC2A88481DC7065779D063CAC
:106AD000AC7BE08390CB19C70862DCC51DDFB8141E
:106AE000C1C8CC03466601479A39CB4525D15AC95E
:106AF000CEB73AE86EDC0AE57B307743F71606F846
:106B0000D3E64F4CBCE02E4681B3D7C518E7CF364D
:106B1000C26F85AE788A6854B77F8B3E4FC96A745E
:106B200077586F0B6F7E02D050D9371784C163ED51
:106B3000039DB8804512FF762551A44ED1F3293923
:106B4000AE1D9BD960039FDCD0960829E08ECB490F
:106B50004AF17EE14323E7321DEAB56C243771F731
:106B6000885662E83F886EC60962B4483F4E4921A4
:106B70009F843D7EA5866DD4A9E041DB4A00ABF140
:106B800054E366F8C8D159978143A9C9674AE467B5
:106B9000091ECEE9B8D417EE2B36A98038A5A46912
:106BA000B5D6B2DC0C3667A8A6FC3687513E8ACE35
:106BB00082386C1C4129EE5D047B0A020D035AC128
:106BC00009B703AFD651921D9858C3130A06EEDCDD
:106BD000A82A9067B746B74649854A7B3EFB601DA9
:106BE000C88D577CBB881610AA441576FAC0065388
:106BF000A245A3B167CE6EBF36D65E46CD3EBA3A49
:106C0000A92486513D0EF7F9F74767F0ABE5214D12
:106C1000215099421E88A5B365F9706189025622F8
:106C200022F63BDEAA7B9279B0C85E2F500B9D798D
:106C30002E0ED8B5307D81FF0267342D7436BBCF60
:106C4000E344C3FE1BC3339649C43746976D685966
:106C500001881DDA490865CEC72AACBFDC7C9BAC35
:106C60003D94A0931A6253818B36C47BA9D7842E9E
:106C7000810B101B4869C5051BAC690890E9F8C079
:106C8000FBA81AF76B623CB508E11379D055C1FC3B
:106C9000521FC81C860C7A7632255630629C43A35C
:106CA0003641AE9B8E5F5313970DFC2BB83EC953F4
:106CB000815D3E5DE8B372D7771E14B35F2E659A8F
:106CC00029268A7960FFF38E6E1408465354A588EE
:106CD00047B6ADE801A8ADACE803B2AF431157AA7F
:106CE0004848CC90CED0D6D0FEDA9760D72BDDDEE8
:106CF00085E9348386622D717512781E2140DF8C00
:106D000035ABA838EE6F78CF9A313E2F3D6327EB35
:106D1000E3F829D1675C52CEC52F9A1BB60849A962
:106D20004FB37F7CD4ED77257A31C0C4E1BA86C9F0
:106D3000A6752947F5C55CF69219F88C4320CF1546
:106D400029C80528B128CA9459A52C36640D0EC847
:106D5000DFFC8B3B9285B35AB86291A6D0838997AA
:106D6000A1BD1A6BA52890BC86596BAA1EE72B42C1
:106D7000DDB32F28B5A6AE626DACC987C9323E3CE3
:106D8000B3727C6960EB684DFBD21915DFD965558C
:106D90007FAFBA0E5D733E0578433D75DF1FA213CA
:106DA0005DBFBB853D6C73EF59969F677EB81CF93C
:106DB000CA8FE5016EC25F49A124A775E1F6B184CF
:106DC000F6BA49AF822C4901A235C8CAE7CCA10C5A
:106DD0005B9BE0FA8576A1AB6599B8664AF14FEA0C
:106DE0005C01B476D8462732C79E19AE4DFE616F5E
:106DF000DA939A664BC9CF78AC79F88829D4FF40EA
:106E0000890B7296AAEAB4192130FBCA796C8A8977
:106E100057E7A8D827DEB2CA2EF963599665CFC1C5
:106E2000D86E726EF808B8D575B2958F94A2638348
:106E3000CF5A19643704224C8A0335542BF9E3499D
:106E4000EB32BC69A10D48B58B0831FD2C2AE65800
:106E500096D88E816DE61CAA75EED5E31C04B41697
:106E6000EC027C607945C321D060A3FF576BCD5EF7
:106E7000A0B13DC228AF46995D6D43D1249466739D
:106E8000B967624FCEA5991742196FF117222D6B82
:106E9000E6D58605DC29662528BED963E10847BC0E
:106EA000CF8B18A9A14FE0E3981D62390AAF22E801
:106EB00002298D181C5A8BA48AF6EE17A966E1AE3A
:106EC000AC7EA6AA6A723CC9F76950BEF9FA197E6F
:106ED00063D069FEB0F351BC7ED9F1E3A8A0E862AB
:106EE000CD10647377548714FBB4594BD7281374AF
:106EF0002C7B31C85E0978A56025E705A2F0DED4B9
:106F0000A2D696B963989C76C390374575B6D109D9
:106F10007027389F9C8B43C40902FBAC57F06E91DD
:106F20000157AA6EE5423BB80100450AF1C8B70D0A
:106F30004E5866C23D6DDEB1F4AC0680234B1FDEB9
:106F4000A8A066B97D87184D8AF5608D29A43941BE
:106F5000076D81399A1F5D780A0FEF15EA843C7737
:106F600053FF1D0D755737F25C27B386FF7F3D2415
:106F7000AB2F4ED6563611383579F65947A1C0C5D4
:106F80008B41CC9945F3792E85AA5FE7D7389A33A0
:106F900093E199E92CA908B602117B28861649CB02
:106FA000E98A9F5266C27E6FA997AEB1ADDA70F3DF
:106FB000BEE2573B8F73FDFA81796951F7CEAE7807
:106FC0002BB25FFF518B24536EA927435C13764786
:106FD0000784B9B02F1BCEA5885E4D16156A753F84
:106FE0006EA947D19745AA7563C42239C71F5F00B0
:106FF000E7F5D2A8928A76FC62A0469C5167494088
:107000006F92672AFA24DFB3C04106A1D3E3654833
:10701000540859304446600B2B187CC415DCC583DA
:107020007841B6A4BA26BE871AD986E0D43D3E98E8
:10703000684FECCB3B2D1366358024EE98362FC07D
:10704000BC568DC2DDC6CC96B0CD704BE6A75D8632
:10705000B04D17686A139CBE8786AAE082625310FF
:10706000DD98F7FDEE496CC9818F5E63465449F2A5
:10707000655DCB8629A1CC1CB47799AC99D4431318
:1070800011B2911A4B092F91C007C96BD4C92E06B2
:107090000C522DAF9A9A6D12AF00C654B59DB743EE
:1070A00031FCC35EEF930B8E46F2272AD37C11137B
:1070B00065B345C99282E092FC4009A6C7B2495A1D
:1070C000962D6AF1C401619C771B92EB8440A91252
:1070D0004EF063C42B6D6DE056BBE315C3B8C329F6
:1070E000345CFBECF64E369C01310C4891C27F9625
:1070F0005DEAF7E2C60D98B85ECCE08F129C04F210
:10710000EE8758269AC1252B214D9A72D14ABF0C81
:107110001877E358ECFA6FFDB71D32A34F412811E1
:107120008144038075E538B1D939FDB7C72FEFF237
:10713000187D4EEEC48BEC8D5BAE1FF23ECE4A0244
:10714000114DE1B4B16A79C3E997F1E24FDC80599E
:10715000A0148AE349B140E52B774EC4F844FE49B8
:1071600075BD3EBF6D6DEBF8EDAB6BC09524FCB704
:10717000EA65C607E58F177490163C5393BD9B0ACA
:107180004F122CBDC415B1D307B30742D8F4FF99F1
:1071900083A5AC851126263CA9442F16A37F7786AC
:1071A00003BD60F002EA89424F7DA4A13A5CABCDF9
:1071B000C110FE37BEC58C90531732B30CFA0FBE08
:1071C000FE6241BBE514F1793A38E84CA1ECA65EC9
:1071D0005FF3449D58977D74022F3FA8AE3A076F26
:1071E000BE6FBDD3038DA7DF3FF764873DC73FFA6E
:1071F000358759ED9D04A7B00FB3B9495B692DF0F0
:1072000031D1C80E36BFB606BC028929B47DFD1F38
:107210004B81D08E1335C8AB66B2E027A6E4656912
:1072200039A211122777A57BB770D8658F28F08E09
:10723000A9C9A5C39432335DB834168DCE438FA04F
:107240000CC410F6DBEF8EBE15D4C893A6DA077F08
:10725000E5C1A7BA2F736F636C6721162389AE2926
:107260004291942577CB78B9FFEBD61BA8D2FAB51B
:10727000B157C065E58433F2A411BBA7F33569C7E4
:10728000AE7FE7144EB40A7D2BFB84A89010A66451
:10729000887AB717A0D74CE2940EC6EA46D9B8D779
:1072A00080F1A40006837512CCB7AA5B7F367DF708
:1072B000A2F8D0311E2260D9F2126B42FD9D4D56CC
:1072C000FFA31534CFCA8DEDFFD27CFBC62D714EC6
:1072D000827163A302890E895FBFED13D54EF80A50
:1072E000C0C97F5E3A522DB38648907F04E2A694CF
:1072F000779FF42BBD1A4F966A86BC383376EF9B86
:10730000F8660B94A3BFCFC651273DB307C787D7F5
:1073100060F368EC019D8BAC0E6FDF48DEE0A43CAF
:107320000681283C165EC6659DA69FA7B0CD58F184
:1073300012FE55354DF4A6A6E8691D454D72AB68A1
:107340002AA79A7C468A6DF906D296E6A7A7672BEC
:10735000DFB9F6C17083A3C7AED3A75104A834E048
:10736000662AB001E5F6CBAA2A374BFBB4040374B6
:107370002FD7456105A917369CC58A7AAEEE22C47F
:10738000422F1A8D5B3DA7E2DC75FDF59DB60534F5
:1073900039EA8C624EC85DDCBC0F9CDA318497A65A
:1073A0006FD93B1A5B4FFC88598EFEF213184F5A67
:1073B0004FEEBCAE68354D563FF6A56B0D3F43A86A
:1073C00038EAA0872C34718238CE046BDB26DEDCF1
:1073D000161FF28B51693EDA444670C13BB4BA7E47
:1073E00036AE1A98FB1657D3C2EDDE40FDAA541FE5
:1073F000FE0000013A8B56B79299641F2BD4E8EE39
:10740000165800812E2A739B94857188077E03A0ED
:10741000026F512535AC34D6448193E50995C9E313
:10742000D008E82BA0E663021BD739B4227842AD1E
:107430002C41C5EBA21C3715015B048A97E78887AE
:107440001DC78FF921D30BAC24B0446B310FB54E5F
:1074500040A90DD9124035570B4C0B4D1619672812
:1074600030C5775E42EF75C810A76AD79E6EDC2FD5
:10747000D95BAA106AB2670EAAF235E2353DE6760C
:1074800024AEB102A87449E59DA91433D09F8C4B5A
:10749000CF84F8E3F8690865170A6B132FAF3148FA
:1074A0002DF987B8E8AB2851EB45C93A90F7CFF3EF
:1074B0005A6A084FCDA7CC0050BC06496263D3720C
:1074C000CB76E426D308959C94D824B082913F3C97
:1074D000179300F8DA3929C0843D708FC3D12B4F40
:1074E000D4BA1FF47793EBD1F8FEF49828A68A6AF1
:1074F0000258933D308A0E41334127750E4DC72700
:1075000009049E1B25A77CA9EB65491BD35B26704C
:1075100090612B9CCCBA820AFF1BB65B89FAB8EB50
:107520002457B25D80CAB786E6196395D4868773FF
:10753000FDA0B5DDCCF3389EA61EC6F0800BFBEF98
:107540000163FF70FB86BD946BD8C55024302AAE12
:107550007D30162945C19D7D1C4BF9C784B8C5B93E
:10756000E2C70CC20B94E9170BD131C0C18020CC0B
:10757000E7A69DB040B7C6268B5B3C6B6662F77290
:107580003864AE67B28B248AE6982DD844B5B89398
:10759000F985EF7373DD44E8F4CB7F7066C6D6E6F9
:1075A000ECD30A4C26DF212DBBF2DE689E8EBCCCCC
:1075B0006F30983B2A0F4CAD8109F55D883332332B
:1075C00057828618445ECBB1FFE54C03CF8BC4478E
:1075D000D0509ED8568436B4FE7A4450B57C0DCB3C
:1075E0000F45870E9FF2154A89C7FF03F143DD2C33
:1075F000417157A06139B507E479834B2E370339C0
:10760000BD17B0F9982D51635DD5D1B11FED015271
:1076100044C5E3142F156C368622D3D13BDEE795A3
:10762000F9C73F1F30264B4818BF10A2EF0E572650
:10763000E9127C5DFE95B7881A5F5BAA6DA5C8014B
:10764000B68F2C30D8655F487D3A63D44C2AE91B4D
:10765000C22F7F62A7DBAF984CC412D51559EB94AB
:10766000E867835E66358D01DD33866D6C73E41FDC
:10767000A763AF86D2E8A7B1B6431DF46231C3E574
:1076800080EB9E77C71285CEDA5E9B5C7157565EA3
:1076900007DEBDA7DA9B959B5E7C68ACFD9AAD12B8
:1076A0003AD4818B6834465F9236AF4C0EF355085E
:1076B000B5F0FAF47BB877095448EBEA9A62476F61
:1076C0008D3DC26AFD69D11E951B0F84EAA6831108
:1076D000406E4611B9FDB49F759566EB04EC2238F7
:1076E0009BDFC4FBE15F1D793B3CAE19F4517AE3AB
:1076F0009323293057AAE937E9D7EB9BDC45E92DDD
:10770000F47786FF1DD71B3B67BEC7FDE1928E460F
:10771000E98064E6B062ED0347B63D19D95DBC620D
:107720009C0819443BFB558AF838431A374FA1642B
:107730006D2A41FA5115478A5019CC358F4869AEE8
:107740001F55EE24BC1C75DA4406F3180BB6E5BCD5
:107750005E43D436D1D70498615CC917ADC21E868A
:1077600045C68960130169B0D0F5B0289F60B81193
:10777000447B5742A39CBA515EAE2EC4D35FAB5B31
:10778000ED4908DC0CBECF4F9CD436B27AA2660A13
:107790006DF3A28D7B5E28C9B49C962C88D9D95BE9
:1077A0002F485669DF1C64C3C2E6631E93D3F08F73
:1077B000121AC6D1BF84EB2B2CC1F94ED0C3401B8B
:1077C000F5736685848D690D4A556BD80BA1D1A4DC
:1077D0009E6A5D2F0DFA765DE6539229751B59F965
:1077E0002E99DDB659C23ACF4126A2A3891A8548FF
:1077F000957B6EBFF3CE95513B3F3DB3E0A5D3C023
:10780000A84647B8F3FCD04CCA6F773BDA4D7BFBF8
:10781000D4FE1904B2AF3660018548B012BC3D8574
:1078200056E2DF096D829CB859AF0CADBE89FF1CD2
:107830007B1F4A757BEB308EEA02BDD76C042E3F6E
:10784000EAD86849FDB6AF63C66AD11A09F91C5770
:10785000F23A6CF24E2A9EC1AB517C3F62655D7E6E
:107860008F5071E0F70C5AEA93AA988610D084F6EC
:10787000C588F2D04F4F5A529A0FE1E0A74ABC1781
:107880003665981D0B03EE2301CFFC31BD864D0DEF
:107890008A82C6FF67207BF8565889A127BEDE93EF
:1078A0004BEC5067D6AA81F3C47A1002E485DBDA88
:1078B0002CB9FFED16D9EAA7CF9DBB700234E13A8F
:1078C00073198022F3B166C3E09D98369DB668C5F2
:1078D0002A4ABACC24E467A1868C9C3CD6FDE6C13A
:1078E0007B7CFF0AB9552E8E31D5067E1199E34A6D
:1078F000512DEC603938DB493FBBD43FE400DA3E20
:1079000074B807F95C7E111B433C2776A415ECA0E4
:10791000B2DF69FA6B992251462EF396714D7AAC1B
:107920007CB6B6638F22720CF5278CFEE23279EEBC
:10793000A1592764E5F16A1F947C7C820D36B68CD0
:107940009E71D566F39BBE43D98FE4BBD602F9B5D1
:1079500057CC449C6A640E5483837D0F89801F79C1
:107960005B46B23F11F5E992DC10A5EC96DC021003
:10797000C5FE853AC18469E98D8EC9596912D93B22
:1079800015A85B66DDC7DD358BE2A157343D8EB6A9
:10799000F0FB7A6A95E2E4C193164088828EA6B520
:1079A000B89EEBD2E39B1C0B9F53B29ED3DC7EB1FF
:1079B000650BE6261A32816EA8CE2B3C947477A410
:1079C000C8E1866D56CC985648EE83A1C76B1F164A
:1079D000E0D133D891906E22FB5BBB960D6E29A847
:1079E000C08806BB9207F53DD533B77A93F774C6C6
:1079F000911ECCB94896304673945B4B7204EA9A58
:107A0000E85549EDE032629541CDCAA5CC03483333
:107A10005947D8A611ED2DA9016F28115729D8B2C1
:107A200084F59DB9C6D8B6F6835B7402659B010BDD
:107A3000FC6BD38FAAF81787EAF54370C723E68C4F
:107A4000EFD0D03F0D8A12AB6108D85DDC04616DC8
:107A5000FC0C927063690D04E160C7C966DA764078
:107A60005FA4B46A79720F2839FFE76BF28F9384B1
:107A7000FA758FE3B688A3DC02A55EDF9CD2CC72D8
:107A80007EE8831677C8809BE214B97F1CD9AC7F4F
:107A9000152CF185F05CB403B989A52C393A5953FA
:107AA0000B15C67426370E9A17A3DBB5AB074296A3
:107AB0002A16A8D781C72760183C37700B8CF79F10
:107AC000F6CBF35E8F70F74E8F815CBB973FCB1781
:107AD0004A1DC133EBE19B7AED4E15698FBEB1941F
:107AE0003148FC8FAB295112946B03CB1AFD61D145
:107AF000720F5D302CB9666D883857D398CE93E5F8
:107B00000642BAEDB52AF1A41807DCBDEDD1025644
:107B100018A68046404DDD7B8B482C82588B7D68B3
:107B20003588F9F50944D97127EDDEF1CA2E4D2AC1
:107B3000D706EC9461AAD967061D1212FC8EA5E443
:107B40002AAEB1E021CD950FCF214F80FA82C7F345
:107B50002466C1156D20B137FC2BE129CE02389384
:107B600043A30180126174317869F8066390A774A9
:107B7000B114E2149B9DDC9ABC3F916A4C560E6690
:107B8000B0EEAE991F7BC132275AEF01A96F46367E
:107B9000B9BB47D27396430B82722CC1D83D1F806C
:107BA0009743A08CB5EDAA3643DD86F8C39A0B66E1
:107BB000911F86E090A52E2D18198C270FE6E24F15
:107BC0000755F94E238F6EFA2ADA110AE86780C941
:107BD000B75875973B0E112EB23197890E2CCC3DBC
:107BE00000A286795BC0B900F60508BA6640C06895
:107BF000121A1AE50DE7C064865E382280444951A6
:107C0000DB76BA4B3024141B7A78000F7CF97F1E88
:107C1000B9942ADEDC7DDA4829566F597A82274BDF
:107C2000811775A5D0C1CDA786DCE9811B644F4DB6
:107C30000A4C21A35036EDBA5E48914D44F0A8118C
:107C4000BF5FD9ECA5374E02BA8A208EE8DBA2725C
:107C5000AEB5E42B8ABA439523738914F32BB7810D
:107C600058764038375A4E5F274530A12A8EFF405C
:107C7000C5B603A7A98DAAD19C955CAB89DA527CC5
:107C80005327D7646843479DD11280FFE0A8E38C57
:107C9000D62863DFBCE8A2EDBEA2439F1AE0945D44
:107CA0004BDC1A11AECF2EBDBA8CBE023EC2BC1F39
:107CB0009E3833E8398F0D6DE6B9A7194DC3A6EF8D
:107CC000985D65717709784D9C99E626C5817A049F
:107CD000EDC465A56A142566B62F58DAF1D1E8E33C
:107CE000E205A3BB7DA41C44185CE7060E9A62EC77
:107CF000507B6F087C3FC9FA7B0EF5A4BB6563C15E
:107D0000BBEE2DAEBEF9188EADA293C5FD9E7415C7
:107D1000169FA2742B03046B69DFC87D5FADB14A67
:107D2000EEB45A5E6C0C15903A03B070623A475448
:107D300016424A8A2FAD987F2EFA0130952B8295F4
:107D4000C7F2AF77AB12AB3BF4FD559181FC272A0C
:107D50008FF40174B0B1ABD041D0F17289B4E78D2A
:107D60002B52B76DA74899345CE551024BD450C7EC
:107D70007481D58160D8F5806AC45C03D9FDBED614
:107D8000B2F3CA4708A757010494869C76C388D3E8
:107D90007A4E08CB6672B8C7B43DDE3862E4DE2F97
:107DA000CFCFF5412E0BCFD8B64908CF64B687EBBD
:107DB000F562369787A1AA37921E69DA6B3989F383
:107DC0006F35A309BCA63E29ED87CCB9348EB8C85F
:107DD000D4491B5DD92D4E36E6A8EA52E804388412
:107DE000EE9AAD1AD49CBBF40AA00ED56C2F0ED817
:107DF000AF47E1F903FD3C1F67782F5BA85276344B
:107E00005A73A7276EAB48BD3489E5EDE45CAF0536
:107E100032800873726B71DCD9267C8A058A6EAF5A
:107E2000B73F7AED0C2CB8AE1E92E5CA5F65941E82
:107E30007FFBFFF9032F993C243AC74CDBB9BF0DF8
:107E4000A36040F9FDB120BE3D295BC2362837A8AA
:107E500059376098C0C048F86807B6B0C552D83ADC
:107E60007F8744243A64A0CE7E52A9DCF5862A227C
:107E7000F8FB3E95CE12F6338A57C485720A6A51D2
:107E8000FF73E195CD6425745999C16AF005785363
:107E90003ED39B9E172F80BC4D45DDA23C583755E5
:107EA0004A33582291D9242C0C954465C7A77CAD40
:107EB000514DA95D67363953F9A844625848656841
:107EC000AD97A0BAE47003EC636CE8D7CF0F0396CC
:107ED000956408A4923FEC2D4A908E7063E02ACC02
:107EE000C61C4A5623412CC8C0DC9B772037C6A845
:107EF000291B35F8856AFF4CEF05F3B9210334FDE2
:107F00006BF5B958BC91E62EAE26A8831BEC0D6527
:107F1000B6903E50AFFD8AD99496C077E7F847A354
:107F2000E8FC3620B9BCE9E8E7021F98AB56623D91
:107F300058FDB1B6C8763B42CE3555E7F0116ED04C
:107F400046713187825C95365D5BFA939A8AAA26E0
:107F5000AAA0622201131CA4C845B2AD7EE1DB4495
:107F6000F1B64A55C395FABEF1B60F686541F047C0
:107F7000A5D4DA91CE8ACF043CEBC44DAA1BA89FAE
:107F80007077E4FAD0237EF011F1D270D2BB39E0E1
:107F900035D8EA1046E4F08ED84D713D686587D932
:107FA0005AB0F4E9435C5BD517E0B3BED1BAE574CF
:107FB0002D669BC787BF4BEEE31E3AF5F864D821C8
:107FC00095AFD537A7385B012BDCD9985F29AA8CF0
:107FD000376C0AD73F6FF2430B2CCBFCBB40D9E187
:107FE00077CFAC45176836ED84C9DDF4A9E6864540
:107FF000E2200A3E6CFBC67195BE3FD3BED4F3C4EB
:10800000B624D966C2555A9CCEBBD4740EB1A5AC69
:10801000A9ACE506701033C30541E8FD703AC0FA1B
:108020007F6F6036E9D1F41860DCC198FD81CCFC2B
:108030009AB14C15FA5219C904B648AA988CE1793C
:1080400015882235CA2F4DD19605FBA8EBA461D621
:10805000803ED1A73D44ED4920A31F59991586D6EE
:108060005626AEDFBE049A19ACBDCE012BE2B65A3D
:10807000CE80102E34E21097B7C775CA4C00D6DCFC
:1080800074ADA2F3D7BB7359FA6018A49ACBB5B9F3
:10809000FC6B19A134C619AABD400A6C13D39BB658
:1080A0006BD5E7D471797D501669062BE1298428B8
:1080B0006585A6DF9510D3F9CC3429DD3854A62D7B
:1080C0006A4036CB4ECFA70018EDEDC46541FF8A5C
:1080D000EDC33C994D66C459BAE5E5AF494E9E0BD8
:1080E00038616D67ADD991A4B1A3910AA86E431D03
:1080F000B9613F1BFB5786D116AD8A850686F83BD2
:108100002DB39742E975E93FC4EAD17B76B7705049
:108110006EDAE99CEAC4DC8ADCD31A7FCDBC5387D3
:1081200012CD28F7D3A89C9C5119D3A01A0D2AA3CD
:10813000EEC7F75FD2AAD71C38BAAF24511B08424A
:10814000E3C9E0115D25EC70949FEB1E7A412B474B
:108150007AA2AE75E64C6AF3E86D028011A4ADA276
:10816000C49A0A48C9F88407CAD4AE062E2673BB3F
:1081700072525258D8AF9115B01A006AAE5C229A6A
:1081800081BD2D98495445D5B6C7E8EE8A4E2432B4
:1081900015ED6E7836096109052047D8879E1F26A0
:1081A00097389D8F3A9D7494A23D79C4D2550F2C77
:1081B0001422361543D804CDFEC6914CE682139E98
:1081C0001FE1D39C1DFE392FDEEB76714527AD985C
:1081D0009BF0AD38CF63B9969ADF98997DCB7E5FDF
:1081E000A459026181248A6329C3CDF3E7CFFE69D4
:1081F0006DBD4BEE4DA134AE6A36D028392CF9E571
:108200001BF65D90D6450D170A360A5932A1955CCA
:10821000171F385997A61E02829ADAC6F0CE732627
:108220007085DA588A247E7DD34A7EF29DE4D97621
:108230002405953E84AE39416A0FE9A796D4C90D4D
:10824000AED3BE657C0BA927251D3E8C094C854409
:10825000F40477DF997EAFA82A99EA1ED8F928F1AD
:108260009352988B9138DDC44359C315513CA9C32F
:108270004420A9336BB1DBF15499F701E2C9D42250
:108280004E89D1DC5DCA5ED2843AB4B8DD7B3BFE58
:1082900094F32A35269A390ED72A03726693A4805E
:1082A0009D0C53D8DD243791CDAE632150DD8C1F5A
:1082B000D2FFF24F4EF24637314C105BF980F5A7F2
:1082C000B3539EAD5AAC68F3BF64251A53A003762E
:1082D000697ACA53ACD263FB7B21F4CE5DE886A5F4
:1082E0007C9E78ACF90BAD2DBD9745DA9993D1F50D
:1082F000091927CE39F9F4ABA9E1351D864833B207
:1083000098A1EB227843AB165D2691150DD5B97077
:108310009187C0AA58D8FBCD5819601A3CAA07B952
:1083200037FD0EC5E185F7D4583F8F424E856D4924
:10833000211FA4157192F55CA166048072D0BD8ED8
:108340009D4B3A997624C96013F35F4C0126DFC830
:108350000DABD2D4F844611DD363A9E4AF0B47B28F
:108360009FFC7683771FFE6D141661ABCBDDBFA13A
:10837000C6E376DAF5CA556BBA3D427B1261558C7D
:10838000B1B74D0B79FAE455ECB7D50F52E6B2B55B
:10839000DF92F3AE768317970FD1F1BEF8DB263765
:1083A00047F31C745059BD95A06671E6C75599BE38
:1083B00071E3579116E789E6FF91E751EDEA2EC484
:1083C0007377BB30C6EC66AC1EB91E57FD20FA2988
:1083D000E46D7B9F0912198CD6E5C19FC1CA6571F6
:1083E00004ABA2E17B31644C370C14AF6073904254
:1083F000A99934DEA89117C585D09F16242FE19A3C
:10840000B1EEC569A222BF496B763705C949D1A330
:10841000A1B9B1F4C490DF95EC01B29754177ED1A5
:108420007D64653E056153D3F590D56BF82C5FBC38
:10843000D08416F3D3980669C026960E7D9DC0E7BA
:10844000BD73D1664A3BFB6F2A90C5C488BF0791B4
:10845000C546B0AE1269CCE02498CEE3FB6EA08195
:1084600027CF3A936D759AE5038C92F6370F87FF05
:108470008A951E76C1431634B3A557A2F027603DF6
:1084800011593AD116CD7AFD04F940879EA15EB804
:10849000B651852685EDC37CD99EF56040DF9EEF01
:1084A0008ECA5161EA5A2E765EDC427715A044E40A
:1084B00044546A065C7B2400F8E1E2E1C38D00735A
:1084C000F7F45761D265E3482E284026F2D17C416B
:1084D000540F0A0CD895B4FBABFC39FBF0D810AAAA
:1084E0009377EC389EC73D4191A250AA7BF902A533
:1084F000CC497706D62221AF9362AAB9BF1516845C
:10850000B9585F13BFBDD0936B8E59AD10BB4D3EB4
:1085100022277E98497C80BC769F54A630F7F7D3FB
:10852000F50FDA26B57EB197DC094611736FB7CD2A
:1085300090AFE1A8128682A39931CF4BA07718B5EE
:10854000D5F0CED825CCB7CE4F6F2DCF626A6471EF
:108550006269870BDAEE6E0706F7A81D1E67E953FE
:108560000C34228629AC14EE2355204BB9EC79A8A3
:1085700013C93BF9150E78EBE4765D33A240C5EDE7
:10858000A22A0E90AC6247610F0ED97AEE21EEDF7F
:108590006671F6515659119D73707454A4FE57704C
:1085A0007A31C860FAC34BD9D31414C56FA0514CAB
:1085B000EFB0A520DFD8F0006863D843EA0214D1F9
:1085C00034F295FC911B76CD341453B55923F6241F
:1085D000B245B5DAB1B1E287A68DCD8D3FF8BCA02A
:1085E00038886B1386B923898646B25851537E75F5
:1085F000D56DE1E6131D0B4348EDCCD42DF76FE0AC
:1086000070CE4B120A28D011F16F4543152DD318A7
:108610008314DF95809916649D1164EEAB10FC14F1
:1086200050BB4E89CFAAE5077E5717C5C5CFBEC040
:108630008AC1D5E446295FCC4DB1AF63DB488CFAE3
:10864000A68C4B970216A09E9B122FD471898E97F1
:10865000B2FFB2C103AD9E03F7830A89BBE49A7EE1
:10866000C258EC91415F4250DBCB40E81B808B76D7
:108670000BEBB17E3DFBE4080EE422FD37BF6AB18F
:10868000419D71BC14C419CEAE42FE27AA21B9C6C1
:10869000D3973B7291D35352E746C44A73AEDCD6AC
:1086A000689927A992AD59828DE8981E9B9345B58C
:1086B000B61420BA833D5F28FC02086EDBB289B095
:1086C0007368ABB5CC5C4103C5005CC4B6A3E67F60
:1086D00032A17A64E6AE596396B7F07A01A5003309
:1086E000A8059385DC039B2E6C73336E38F280A053
:1086F000B64AF1C906AD8EE9E0178E22C7A78B698D
:108700008C6C9989D8674D35B2852FEA4CABE73E22
:10871000E48351DA5283CEE2AE205B70E6A8FD0816
:10872000F18B1E39666B738E75C1A5B805D7CB1258
:1087300078CFD47231C09A12EF96FEF18B05CC003F
:10874000E918B987351122060B57D2182C1A30E5D3
:10875000FB83D644A8ACFDAF91AE8F8EFA1A161BE0
:10876000768FA340B22F981ECA8B8857C7AB8CB8A0
:10877000587148C895880BDAF604C263E333769DD6
:108780002DF00F20647415BEEEDF48171F6AA35A40
:10879000F7AECC60DDA4835F68BA1838AC27BA9610
:1087A000BC28785A99FF89BFA52172498D9CF4FD98
:1087B00041874C4E66C0F21DEBFCDDB1361C3A0E13
:1087C00067731FFAC0FB9CE33107AABAF2C53907E9
:1087D0009FB29F12ADF352E18173546C7766968617
:1087E000FECF22A0A57ABAAD22402D0F9CA607018C
:1087F000A9B6A19A8B523EA0DD9A3005DF991CB92B
:10880000DA7E26CEB9E4A1B8BF90F2001ACFBC033D
:108810007532CEE167052C1124D0510374023CE778
:10882000DBA467FEDEA708C56801A53E534798EBA9
:10883000CCA6694784D694FB418EA7073A0E5A6AA4
:10884000FDCD14F6C1E2141B2815E71DA10E5CCD69
:10885000D9D4E8AC6C5C431409A159CF61177FD41B
:108860005F818A871B45C4F5EFA5ACCDE1A1AB596B
:10887000B742A01F53692328636BD3A8F5A05A5EA3
:10888000397EAA8B97364DD2B6BDE0DBAA49921F3E
:10889000FAB04230DAF116F31A85550B07F341F9B5
:1088A0001B8D3C4CDDA0EA067A7EEB47F8009EBBB0
:1088B00019CAD71E6A31083EE2CC06A451F1AA7E3D
:1088C00054FB68D5F5F1C9A7AF412293954E2F9976
:1088D000E02E2D13F03526459014A5326C10A234ED
:1088E0006E2ADE85D859DD9D2B4CD8EF21DE6865D8
:1088F0002E77B21C564C50BF6788B783462ABD1DE1
:1089000042CF22A1DF918E4411E648B187EDDB36DC
:108910000FB9F0C3A6F9B0A4FCEF80E018472B35DF
:10892000AF8B4C868C4102CF55F25DBE1659D844B0
:10893000F9158E4D570947A1D28D2DD5ACF9C89C9C
:108940009183B6FAB95F5A3EEE4D780102567880AF
:10895000C0DB092C4E4C1B677350B6BA5C0F59E054
:108960004D36FA02431293D0E1A73939DAB4A05058
:10897000C1CA160BCEFD308B3714DB0BF185637744
:10898000669EC58E7D9B75B2A080FB8F37435801D4
:1089900029C577D00F8675433A231E197EA6D2F0DB
:1089A000F1D204D567514DAD717533863454FC4016
:1089B000DA19B655DA948F0FC06336FA7E087B2E2B
:1089C0000D55912EAA0775F4B5F3D24A08E9A41FF4
:1089D0001C2F29D2E50EC5F0662596AC2E13F27435
:1089E0008104E986B65269068584E58FC43BE402BA
:1089F0001EF95727312138FE67B6189EC43AA1F8F0
:108A000048C23D268CAC946BC90FE31F1306862623
:108A1000B8DEC85A64724E281E4821B44CC7780983
:108A2000EBA5F80281B17C94D6B15CC13C4934FF1E
:108A300098F3F84BDC01469E6398AFD02AB699E8CC
:108A4000D0633590026E5BAD98E2DE7536FB447FF5
:108A500094B601A7DF06E9EC4D2AE1D166D4DEDE4B
:108A60006A98351D1C778249ECED67ADF53A6BC00D
:108A700025DD25D8B53D15484881C95198C0A3C208
:108A8000D3A0D445FF4B6BA843F935CAE14D5682BC
:108A9000DBBE8D5F53008AF2C5D4DADEC2F8DA9508
:108AA0009E09588FB3FC322410E2DD9B2560602FB5
:108AB00062E4737B0083E7298983A0C3C9D8EAE015
:108AC000959F81CB78A23F4FE1C18407ADFE03C3E0
:108AD000FBAB3A4DB14A8722407260325A3D536730
:108AE000B2FF21AF745616ADDB38FFAA5DDC879D5F
:108AF000F21D84A36C5E94FC6323F43EBBFA61E533
:108B00000038ED8A2998F426EF3233E014869897DE
:108B10002E9BE87EFB017E431A5B4021EC5878A136
:108B2000425A9A2EBF412D9897617B135BC85BEA2E
:108B3000DCF478BDBEE3D585291EB7D8A1FB5F2044
:108B40001C27C18BECB72E7863684AFE8FD2F35393
:108B5000725B2769D56BDC4F6F7CD52F277F844DE7
:108B60004727CD9787467E6E1897E7A550EA0F53A3
:108B70003B3DDB17D3C4E5672EAEEAACA5914B02B3
:108B8000203341CEBA4A4B58009DF89111AC52782F
:108B900020068A29F62CA18864FCA837481EBCEA66
:108BA000EAA8F640A799393564DB9C240248E94CD1
:108BB0006F40CB1EEB979F381983FBBAA80AAC6AAB
:108BC00046A1FEDB1021651F78A7D690D521443A37
:108BD00051D46BB88552A1BA1DFFD439C883AEFBFE
:108BE0002AEFCFC7E45A68D43C6443765509BCB336
:108BF00050168FB6325C65093F4D925B534F9439E6
:108C0000FE4AA4AAD1447C022DC0B794D929236579
:108C1000C54891D39F5810F49AC3ECF5566CA180C7
:108C20000EAF5724541CAB2F64EFA13E0D08E6563F
:108C300028C20AF95D39298B4E523E816BE74A28DA
:108C4000E1CC52FFDC8957904AB89F1ECC1CC1E88A
:108C5000BEEA81D4431512E01E134BAEDC393D8EC3
:108C6000B7FCA6DEEACD0DBCEF728EE783768AB242
:108C7000CDC7FE0719124ECCC83A952DEA5AFBAD66
:108C800098BE96BD22ED5E72563ACA245E2F8905C3
:108C9000A52160484C22BB89E0B49F8202A956B14D
:108CA000DD081D44466D6E5F48B2AFA93ADD3FC195
:108CB00026D57C6A6301F80D4A335D476D20583034
:108CC0003A05BCCDE0B8A1E1B74B1495AF07E6E794
:108CD00057C7047090718E935D779285272938521B
:108CE000E9A94D8C9EE7AA8AC77FEFF16653F63457
:108CF000BE0B26386B04FB39153BCB95D5B283F9F7
:108D0000C25B03670CE7D2E559FC2E2F7C3EA6E43C
:108D1000E26EEA33A5B5DCB39D3207AC0A1D5E18DE
:108D2000D131D71B34A3557C4F0F061069D1DE0615
:108D30006AB7FF392F04E1F3D6C1026AAE6262BBA3
:108D4000F2058E28D76DDF74D270B17BADCEE62FE1
:108D50000C38712C2C052CFF7390ABDBA85F68D707
:108D6000FEECF66018FF11E190D999B9CAB620401F
:108D7000750E4AFEEF2B8D5F0186E4F55A266B01D6
:108D80002619E26797ECBA98EF0905C91FFE179DEF
:108D90009C827C657FB8F4C8080AB6473B7776B7F3
:108DA000290A4ACDEBF8E3A91A7C4A77EA63C84955
:108DB00020F659979685376166EEFDED4A4098702A
:108DC000F8B1D7DF08AA3D683FECFC8A814967E328
:108DD000AF799A7FD86987F6382D4E39E6DB7DBEAC
:108DE000A2F897414D73FA240AB47B50074A420710
:108DF00050AE4029FEFDE891C33D777AC3690D7CF2
:108E00007C2A11F0138A2B78F57E541A076635AA4E
:108E1000CD6F030FB83753883A16F602DC8B2E8BD2
:108E20007DABB7918756892D9FA9ABC8AFA2ECC681
:108E3000B0941C78D9138F7E6F6FB0A8F297A8A654
:108E4000CCD15D274FD06CB42C4FBDE625DC69C476
:108E50001079F09A59B2843A389460645ACC63819C
:108E60008AE5E88042DCC56A661228055AA52AC749
:108E70002B810B8D1637AFBE6AC43ABAA8FDE6DE69
:108E80006D2082F99E860A36C0F9E98881D86AEA9F
:108E900011BB50844A76612045C8EF81026DD6CE61
:108EA000BB27E2F6C16F7D4E181AB21E87E2E92495
:108EB0003B5ECD847ACBD7CA6D62C252EAB065738D
:108EC0004B363CBE5D417F9840AFBB7D1B4BD1B55F
:108ED0008AEB3DA07D1420405239F2FC1548FC3D40
:108EE0007A1250938F91A886A9BC182F38A1601CC4
:108EF0001C4FF13347BC066CB405486FD30BB7B4B5
:108F00005D9BC2C06617831017767977E4FA20DF7D
:108F10000DC11E299A0114E0518514640ECCE2356E
:108F2000DD93FF36B93A701917C8BA175E377A73EE
:108F3000EF3F9732D0321DEBC78C70ED4E36193DA6
:108F40000F38A40FA46FA296FA4983E5B8B241A2E4
:108F50009BD00B5D2299242523D4A434E43328AB81
:108F60003AA4EDD155960858E84D314047FB90663C
:108F7000A53953C27B309A056567DA593B997296D9
:108F8000357B75F4EB1681F436D57ED02ACC4A2495
:108F9000F5F380023E8CBEF1B92B325EDD02B0EB00
:108FA000FEB65503EC5C741121F2262A04DDD86A62
:108FB0007D00E22EFD73FAA11D5A68ED5130562D49
:108FC000E34953C1AE5957021305DEF441BE3A30AE
:108FD000E90C85398A1DB03805048EF34C2C196CC8
:108FE000CA66A87A88E78E75DABA7C9B166D8651B8
:108FF0003C7E53BB5A014B08E3531C0D6EAA52EC46
:10900000D2880148717B8E716C7658E2940A90B0D8
:10901000F3F793DB73DA937E2E34DB1F71183E4136
:109020007E602420A8E54B2678CD53AE2DF31E019B
:109030009A5966E04AFE93A259C67EC8C76CB0B87A
:109040003454907406ECD82A18AAA615CB5682740C
:10905000B4712C413F6AB6F3974A79E1C5A3319EBA
:10906000EACD50D006516F8C456A796860AE77CEF4
:10907000ED65EC65264217920AA4BC3772E96D4C87
:109080000F34B78209273C72AA8551A3B7A6219154
:1090900064BD9930C5CC7D443D6E33D0922D9B226A
:1090A00033502DEDE5066AE4E7032A109ECC87F1E4
:1090B00016051E219C7C8773EA89AECC88368832DF
:1090C000DB1FED2DD5B74133109C9B708026F446F5
:1090D000447D5439628B18D59C6F3FE269B5B9075E
:1090E00068E64B313E7BBA9A00EF4A49F2D8564EB9
:1090F00052697951E49EE1C61ABB2F7B530C7B74F5
:109100004BA3019C2E172C0DF19D1E438665FBBDC4
:109110008F251F11A3383D42A4195E143002BA3FB7
:1091200014B1DF35F68594D03071375ABECED433C2
:10913000D15BEB9ED6C8260B827073BD54867259E4
:109140000C6B1606F54B7541F452F69E9FBC46B16A
:10915000308CC16CA5E4A32332D29A324F381AB2B4
:1091600047F98F6864FB3FF105BD0C939E6C79ABAA
:1091700072FEC823DBB0A72D517D478F5C100481A0
:109180009CE895A737FB4E054FB6B91CDD21D635B7
:1091900070FCF2371D78AF9DF7E73CBFA023B5CD3B
:1091A000F796457298BF9937B710A99CE0F2C36E45
:1091B00083BE03ABB7D1B210FADEA2776B3BFB558F
:1091C000A0F6831FFC89AA8993BFE95B9F21DC710C
:1091D000B4F404584DF62A715F4AAA4C02E48EAFEB
:1091E0007D36DCB9717546057F7B37CC6E0217374B
:1091F000B85A59C37E0004E8D6FB0D7F9C3CDFCBF8
:109200006B1B7818FE210AB00067141EE4DB6D0B9F
:1092100099173683EA42AE9B555C1A574550871D15
:1092200020578EB3FB4C4D80955E2DAC969CF0780C
:109230007F5857423126EEBF202AA3870224E61C1E
:109240003231B6BCC6929A1A151AB27C82A7D25B8A
:10925000BAFC2E6D98A4EB9C45B14A70FBBF433419
:10926000B8F2BA0A0DC334B41C459F407B95F6B1E1
:1092700011801A0EBF3F012D357B21A9C7F25E3B3D
:10928000896C32447E1160283ECDBA739C40B1593E
:109290006BAC2C96EBEC20FF99D672AE85EE4BF7BB
:1092A0005516F5B6C3147A0EA76D44A644FF574B66
:1092B0000D132FCD4A4BBD8F2C9C17598A559CE915
:1092C00025A52F09624704155BB74892DC58614712
:1092D000BD9DD671B849ED6B754AF82A5A4F69376A
:1092E0005CEC5C64F13F1DAB9802DE197C97DB53AC
:1092F000C931D9D79CD3A799CF3357121D951B914C
:109300001F0653FDDCB01D38CA121ECFC2833901BF
:10931000426DAC6A25B3AA35B334A210371557F2A3
:109320009EC1E089D15BBA86C13B923FDB2CD0A2C3
:109330006BF13AC2AE0E10AC8D87CA2F5EE6402CA0
:10934000C27AB699CE14F088FF2D9668F976250773
:109350003E3B5AC932C840CEEE65A43D316AE9228F
:1093600011F14117BF8021DA9D2CA2E8CA6F7E3A25
:109370008ED8DAC3F54B34788A75F28ABB8D81E0DA
:10938000F9C718A822F8406394AFD818F1808D9CD3
:109390008120785420C5EB35CB3BC89A1C7B3A1B07
:1093A0002B12909AB349D40B6C2A2F7DA355610BD5
:1093B0006440EAD556AD65A9C265B29C13AE2E30A5
:1093C000D5476BFFEA1CA842EE20609CFFEEE2D777
:1093D000B04A1C7C8E691F64C9E5ED66FDB9DF5398
:1093E000F931F2FFB707C15980993B1C4C01307D20
:1093F000101FDC72DDB8D2D6D46F4C5C517B8495E3
:109400009B910BF611399FBD9485FF03D4CA9B90A5
:10941000144603314D9197B21756B80BF84197E8AF
:1094200041A933F99A2B2BED1E3AB3B9FB819F81E9
:1094300037C5A9EC9946F5D99D8EE85E9DA9E41241
:109440005751E887A10307CE518C160982E7C291D4
:10945000FEA66E44A79E8BC4470ABB503A16CE7B2D
:10946000446E2FDBD87A4D8CC5FF302E7A8E581E75
:10947000DDF300D1A468E2818AE25B3B6862FCA56F
:109480002832E2F7285EADE62993ED1FBB94C28A2D
:10949000594E50ABE6F898FBF9C5E7034471904E7E
:1094A000D935A180DD413FB2EA53AE8C1D33A72FE1
:1094B00070135DA52232DFFCF4F56CEA794C76A1DD
:1094C000EC25030F546E7134DFA578BF7F50958D66
:1094D0006C395CC448158DB958007095F7CE2C389E
:1094E0005D37F29D640C08D31D3B2D824FEE8265E3
:1094F0006FDFE389C5281D3B389623FBB03362A29A
:10950000AF86D35587C7C84093FB1F290CF8F4E7F3
:10951000F0EF38766FE53B2CB7BA4774DD1CBC081A
:10952000CAE2B622A85FD85AEA0A9F5454DBA8C7F9
:10953000882F2D55FE3793CC5AE5F071EAFC6C93D9
:10954000B895F6D8AB36E6AE6DEB07B21B559E0864
:1095500008AE2671F2B5741998EE87D3625BE74BBB
:10956000624EBDE66D306C07ACDB2253B3C2F0FE39
:1095700068E2A6EF1EDE90B7782686EB61A9159EFD
:109580003F63E09F233EF89F0A8C76BDBA05370BF8
:10959000AE1F8AD4A2B361CA664C24DEBEB50A05EA
:1095A00003F85E3F67232CC83DE4D06AC314CC089F
:1095B000EB56CF3907BBAA4DA2B288FB3FAE7D1D4B
:1095C0003931E5EAA416A5F970609CBAE7106F95E9
:1095D000DDD4C1CB00C81AF502CA6527AF7145BA00
:1095E0001D62C9AEA2D2ACD4B3BC840AA37D0786E7
:1095F000664853586DF58CFAD2CFC6FD5A50110605
:109600002048B61456041E51F4F6B881BD15706793
:1096100016AD0BC3EE9753CB0AF78325B18EAA4242
:10962000194DD7BEF24FC35C36528F95CDF87A07ED
:10963000390A352A03E4B1559F44F80F6775E13ABA
:10964000840B39E0D8CF0586B3A8745F56AEF5D049
:109650003766A484FADBBAE8C6E1B02E513B7FE658
:109660001EA2C7FA5E8730E1FB71FFC2CBA3B35CD9
:109670001A65D2D4B2B8E4BBF5E2BE1F06B467F9EE
:10968000B51BA7953CC142C56605307086D2E7D2AE
:10969000C238F0775A617116C83E1730A22923F2FA
:1096A000318415A4412EE78123ABA4A2F6FDE46624
:1096B000F5686D7CE078601F3300D8DA7DD7E00F65
:1096C0001DDABA4B4A378811A7DA1962C80844D89C
:1096D000A714D3DAC954F68466D0AC81CED83891B9
:1096E000FC98772D28AC41D10C2A36FB8415914883
:1096F000DE387EE764E1BE51687CF269865BFF1F5D
:109700007141D75D7346FA500832DACCE41C03CAC3
:109710004D1938A36F6DF31841031E0AF6BAC1E064
:109720006E29AF85F03AC3CD222DB3D7E1E6C2E46E
:10973000DD431AB8FBF3A64B9AA49496C416426A6A
:109740005828F72E4CCEB714495A6F215142E6BF24
:10975000F416220D8F06E495E0C438424A882A3A6E
:10976000FB24E8B9FA62533A1F18BF1B09E5C1444C
:1097700000CBB3BA0E63CB7925DAF12ED9E701B568
:10978000DF360B892DD63ABB3FC2691DB243456017
:10979000EB2EBF24FEF546856830547DA9C74909E4
:1097A000F1001FA698BA6C897CFFDCDD42E9BBF3AF
:1097B0002F3C0B2A225FE1A6C751B1149B530B5CCF
:1097C00079CD01906896E2DC0950F5A4DCAB2287E4
:1097D000B1FFA39C04C7748319D2130A4C58ECD16F
:1097E00067587B84590A0554C8B1C5C2DA7AAFCE2E
:1097F0003C1D5FCE9AADF3B3016B2E937B3FCF7AC6
:109800009BB8EFDBFC1A981C1A477E29BC25C3B90C
:10981000D6E196EDC4A84B9661B4DDF5C2B0688878
:109820007E5AA1BA8BBF7DC58F77849CEB1A36DE3A
:10983000477C49796926914D4EB6850532193676B1
:1098400024ACD5EC9986E9C970CAA8BDCB1B1BA175
:109850005E0D63D4D1DF3F474CE512CBF72FCDF738
:10986000B9D7255BE41990C0CD82EB40D114ADADE2
:109870005C9A6D632BD1724201E5152A7C66D9850D
:109880001C2458D8431D7A76F7D129CC1CB1443218
:109890004AFF0763ACB449868730A6312CACD29C12
:1098A000EAB9BA74B673A23378F46FCD45105A97FB
:1098B0003D762DF7BE79F01B80A7EBA0DEFC94BCB3
:1098C0005295DCDF4C9275D9FBE6FFE1189070F2FF
:1098D000845B729E637618B0B656E1C344DAEC95A9
:1098E00041B0367BDA57F0166D9ABB1F877DC7945F
:1098F0000659C637FD2694038211DCE11E0D27228E
:1099000061AA1367C8DE6C80A99F5DA67B3F1249E0
:10991000C794DCCFD6492A7350197B8F49473E46FE
:10992000538FCF19F376E13B68AF8469D8B6AF5156
:10993000E3B725B6D82EF6241998AA0FFCB10B6D03
:109940000A78F414D2C445C4169A9E679E63003206
:109950006839BCCEE6262D880D6B79F244038D2044
:109960001175C5E84AEADC92DAAE0ABD3A5AA11B83
:10997000832C56FEAA17D03CD9EEBEDB217453C609
:10998000AABEAE262F78618DAE3B861BD2A88EBDB7
:1099900031A6642F6773060C95E73A766197B8791C
:1099A000E1C728CF617A74382BDF5C585AB9FAAB1B
:1099B00013F9386A658BA213E6B178A9E60981909C
:1099C0002254B2AE47CFC94D71A33293983B2FA713
:1099D0001C6E3866C989804B652CC49EC1B9C548C8
:1099E000853CFE4808D05227FD4A4EAA0304050ACA
:1099F00008060BFF0209070D010C00FF2025692056
:109A000025692025692D256900202025633A2569CF
:109A100000202020205F5F7C002C006100446973DF
:109A200070206F66660D0A00555345520046004788
:109A300000424547494E0052414400442E4D5900D2
:109A40005052474D0055534552202020006620209B
:109A50000067202000424547494E2020202020005A
:109A600052414420202000442E4D59202020004304
:109A700020202000081C242C4448586C7405000049
:109A800000FFFFFFFF4D000000FFFFFFFF0F000082
:109A900000F4010000040103010201010411040F9C
:109AA000041704160118010000459A00004D9A00A1
:109AB00000519A0000559A00002F9A0000609A0009
:109AC00000679A00006F9A0000409A0000050205A6
:109AD0000804080B08040405010504090809040624
:109AE0000807020602040206010604070103080330
:109AF000040C080D020C0203020C010C040D010DF4
:109B0000080D0408020808070802020704080108F3
:109B100004090209010A080B020A0201080A010AE3
:109B2000040B0102080204100811021002110810AF
:109B30000110041101120212011302130812080F7E
:109B40000812041301130414021401150215081459
:109B50000817081404150115041702170119081A2B
:109B60000219021602190119041A01160816041B1B
:109B7000021B081A0818021A041B011B04180818F3
:109B8000040B042020202020202020202000000082
:109B90000003000000289A00002D9A00002F9A0070
:109BA00000319A00002F9A0000379A00003B9A007B
:099BB000008B5D0000409A0000EA
:00000001FF
